:100000000C94AD070C94D5070C94D5070C94D50728
:100010000C94D5070C94D5070C94D5070C94D507F0
:100020000C94D5070C94D5070C94051A0C94741AEB
:100030000C94D5070C94D5070C94D5070C94D507D0
:100040000C94D5070C94D5070C94D5070C94D507C0
:100050000C94D5070C94D5070C94D5070C94A61CCA
:100060000C94D5070C94D5070C94D5070C94D507A0
:100070000C94D5070C94D5070C94D5070C94D50790
:100080000C94D5070C94D5070C94D5070C94D50780
:100090000C94D5070C94D5070C94D5070C94D50770
:1000A0000C94D5070C94D5070C94D50744617900BE
:1000B00041636374004C6F616E00436170616369FA
:1000C0007479200047756E732000050512151F1501
:1000D0000905082466E766244120596573202042FB
:1000E000204E6F000042726F6F6B6C796E00436F31
:1000F0006E65792049736C616E64004D616E686154
:100100007474656E0043656E7472616C2050617228
:100110006B0047686574746F0042726F6E78000000
:100120004C7564657300537065656400576565645C
:100130000041636964004865726F696E6500436FD2
:100140006361696E65002000200003081F051F1F02
:10015000151B1F11111F110E1F15111F05011F1156
:100160001D1F041F001F0010101F1F041B1F101055
:100170001F061F1F011F1F111F1F05071F311F1FF4
:10018000051B17151D011F011F101F0F100F1F0C3E
:100190001F1B041B071C071915130C121E1F120C22
:1001A0001E12120C121F0C1A14041F052E2A1E1FD9
:1001B000021C001D00201D001F041A011F001E0448
:1001C0001E1E021E1E121E3E120C0C123E1E0206A7
:1001D00014120A020F121E101E0E100E1E081E1AF6
:1001E000041A2E281E1A12161F111F001F001D159B
:1001F0001711151F07041F17151D1F151D01011FBE
:100200001F151F17151F00170000100020100000F9
:10021000030004083E09093E3F25251A1E2121122C
:100220003F21211E3F2525213F0505011E21293A99
:100230003F04043F213F21001021211F3F040A31C8
:100240003F2020203F02023F3F02043F1E21211E8B
:100250003F0909061E21112E3F09093622252519BD
:10026000013F01011F20201F0F10201F3F10103FD2
:100270003B04043B03043807312D2321102A2A3C78
:100280003F2424181C2222141824243F1C2A2A2C20
:10029000047E05014C52523E3F040438243D2000A8
:1002A0004040443D3F081422213F20003E04043ECC
:1002B0003E04023C1C22221C7E22221C1C22227E86
:1002C0003E040204242A2A12021F22201E20201E7D
:1002D0000E10201E3E10103E360808364E50503E7E
:1002E000322A26221E29251E223F200032292926B5
:1002F0001221251A0C0A3F08172525191E25251835
:10030000013905031A25251A0629291E002F000088
:10031000002000004020000000030000000000005A
:10032000003E5B4F5B3E3E6B4F6B3E1C3E7C3E1C7B
:10033000183C7E3C181C577D571C1C5E7F5E1C00C1
:10034000183C1800FFE7C3E7FF0018241800FFE778
:10035000DBE7FF30483A060E2629792926407F053B
:100360000507407F05253F5A3CE73C5A7F3E1C1C51
:1003700008081C1C3E7F14227F22145F5F005F5F11
:1003800006097F017F006689956A606060606094FD
:10039000A2FFA29408047E040810207E2010080802
:1003A0002A1C08081C2A08081E101010100C1E0C0D
:1003B0001E0C30383E3830060E3E0E06000000009F
:1003C0000000005F00000007000700147F147F1486
:1003D000242A7F2A122313086462364956205000CB
:1003E00008070300001C2241000041221C002A1CB7
:1003F0007F1C2A08083E08080080703000080808A2
:100400000808000060600020100804023E514945C1
:100410003E00427F400072494949462141494D33DF
:100420001814127F1027454545393C4A4949314146
:10043000211109073649494936464949291E000014
:100440001400000040340000000814224114141469
:100450001414004122140802015909063E415D5955
:100460004E7C1211127C7F494949363E414141225E
:100470007F4141413E7F494949417F090909013E88
:10048000414151737F0808087F00417F41002040AF
:10049000413F017F081422417F404040407F021CC1
:1004A000027F7F0408107F3E4141413E7F090909D8
:1004B000063E4151215E7F091929462649494932A4
:1004C00003017F01033F4040403F1F2040201F3F6A
:1004D0004038403F631408146303047804036159EF
:1004E000494D43007F414141020408102000414131
:1004F000417F0402010204404040404000030708DD
:100500000020545478407F284444383844444428D8
:10051000384444287F385454541800087E0902187F
:10052000A4A49C787F0804047800447D4000204007
:10053000403D007F1028440000417F40007C04784B
:1005400004787C080404783844444438FC18242493
:100550001818242418FC7C08040408485454542413
:1005600004043F44243C4040207C1C2040201C3C90
:100570004030403C44281028444C9090907C446487
:10058000544C44000836410000007700000041361A
:10059000080002010204023C2623263C1EA1A161A0
:1005A000123A4040207A38545455592155557941D2
:1005B0002154547841215554784020545579400CA9
:1005C0001E5272123955555559395454545939558A
:1005D0005454580000457C410002457D42000145CD
:1005E0007C40F0292429F0F0282528F07C5455453A
:1005F000002054547C547C0A097F493249494932CD
:100600003248484832324A4848303A4141217A3AE1
:1006100042402078009DA0A07D39444444393D40AB
:1006200040403D3C24FF2424487E4943662B2FFC58
:100630002F2BFF0929F620C0887E09032054547906
:10064000410000447D413048484A32384040227AD7
:10065000007A0A0A727D0D19317D2629292F282654
:100660002929292630484D4020380808080808085C
:100670000808382F10C8ACBA2F102834FA00007BB5
:10068000000008142A142222142A140895002200BB
:1006900095AA005500AAAA55AA55AA000000FF0075
:1006A000101010FF00141414FF001010FF00FF10B2
:1006B00010F010F0141414FC001414F700FF0000E4
:1006C000FF00FF1414F404FC141417101F10101F63
:1006D000101F1414141F00101010F0000000001F51
:1006E000101010101F10101010F010000000FF105C
:1006F0001010101010101010FF10000000FF140058
:1007000000FF00FF00001F10170000FC04F4141489
:100710001710171414F404F40000FF00F714141455
:1007200014141414F700F7141414171410101F10D5
:100730001F141414F4141010F010F000001F101FF8
:100740000000001F14000000FC140000F010F01066
:1007500010FF10FF141414FF141010101F000000DD
:1007600000F010FFFFFFFFFFF0F0F0F0F0FFFFFFE1
:100770000000000000FFFF0F0F0F0F0F3844443838
:10078000447C2A2A3E147E02020606027E027E0273
:1007900063554941633844443C04407E201E200692
:1007A000027E020299A5E7A5991C2A492A1C4C72CF
:1007B00001724C304A4D4D303048784830BC625A56
:1007C000463D3E494949007E0101017E2A2A2A2AE6
:1007D0002A44445F444440514A444040444A5140C2
:1007E0000000FF0103E080FF000008086B6B083683
:1007F00012362436060F090F0600001818000000F4
:100800001010003040FF0101001F01011E00191DE2
:100810001712003C3C3C3C0000000000D5F08D1459
:10082000A1C881CFD9F1AF2000F0F89C8E878387D3
:100830008E9CF8F00000FEFF0303030303070EFC89
:10084000F80000FEFF0303030303070EFCF800009B
:10085000FFFF00000000000000FFFF0000FEFF831C
:1008600083838383C7EE7C380000F8FC0E07030304
:1008700003070EFCF800003F7FE0C08080C0E07FEF
:100880003FFFFF01010101010101FFFF0000FFFF28
:100890000C0C0C0C1C3E77E3C100007FFFC0C0C0F5
:1008A000C0C0E0703F1F00001F3F70E0C0C0C0E04C
:1008B000703F1F00007FFFC1C1C1C1C1E3773E1C73
:1008C00000001F3F70E0C0C0C0E0703F1F0000008C
:1008D000000001FFFF010000004861726461737352
:1008E000272063617263617373212100646F6C6CF4
:1008F000617273206F6E204F666669636572007463
:1009000068656D2120596F7520666F756E642000D3
:10091000596F75206B696C6C656420616C6C206F1D
:100920006600596F75206B696C6C6564206F6E652D
:10093000212100002020596F75206D697373656453
:1009400021212100006861766520746F2072756E28
:100950002100616E792067756E732120596F7500D3
:10096000596F7520646F6E27742068617665007416
:1009700068656D2100596F752063616E277420735F
:1009800068616B6500616E20616C6C657921210086
:10099000596F75206C6F7374207468656D20696E73
:1009A00000756E697473206F663A2000596F752068
:1009B000666F756E642000323030206275636B7331
:1009C0003F006D6F726520706F636B657473206696
:1009D0006F72007472656E6368636F61742077690B
:1009E00074680057696C6C20796F75206275792086
:1009F00061206E65770057696C6C20796F75207384
:100A00006D6F6B652069743F006C696B6520676F63
:100A10006F642073747566662121006865726520B5
:100A20007468617420736D656C6C730054686572D2
:100A300065277320736F6D65207765656400646F4B
:100A40006C6C6172733F007370656369616C2066E2
:100A50006F72203430300073617475726461792074
:100A60006E69676874002E3434206D61676E756D31
:100A700020666F72006261726574746120666F72C5
:100A80000034303020646F6C6C6172733F005769C2
:100A90006C6C20796F7520627579206100616674D5
:100AA000657220796F75210064657075746965736E
:100AB0002061726500206F662068697300616E6452
:100AC00020004F66666963657220486172646173D5
:100AD0007300696E2074686520737562776179218F
:100AE00000596F752077657265206D75676765645D
:100AF00000617265206F7574726167656F7573212F
:100B000021212100636F6B65206275737421205071
:100B100072696365730050696773206D6164652055
:100B20006120626967007072696365732121210029
:100B30006174206F7574726167656F75730062759B
:100B400079696E67206865726F696E6500416464DB
:100B50006963747320617265007261696421212187
:100B6000210066726F6D206C617374207765656B10
:100B70002773006368656170206865726F696E65D0
:100B80000050696773206172652073656C6C696ED3
:100B90006700626F74746F6D6564206F75742121D6
:100BA0002100576565642070726963657320686110
:100BB0007665006C756465732121210073656C6C2A
:100BC000696E6720636865617000526976616C20A8
:100BD0006465616C6572732061726500746F646135
:100BE000792100626F72726F776564206D6F6E6538
:100BF0007900596F7520616C72656164790021001C
:100C0000596F7520646F6E27742068617665206166
:100C10006E7900004F6F707321002100596F7520AD
:100C200063616E2774206166666F726400004F6FA7
:100C30007073210021006D6F72652000596F75205F
:100C400063616E277420636172727900004F6F7068
:100C5000732100596F7527726520646561642121D5
:100C6000006265656E206869742100596F7527768A
:100C700065006D69737365642121005468657900AE
:100C8000796F752121200054686579277265206687
:100C90006972696E672061740041204669676874F3
:100CA0002020422052756E004552524F5220004182
:100CB0006D7400536176696E677300596F75206FAC
:100CC000776500596F7520686176650057697468AB
:100CD00064726177204D6F6E6579004465706F7343
:100CE0006974204D6F6E657900426F72726F772064
:100CF0004D6F6E657900506179204C6F616E000018
:100D00000051747900507269636500436F737473A6
:100D100000596F7520686176650053656C6C200022
:100D20004275792000000075703F00646F63746F36
:100D30007220746F2073657720796F7500646F6C13
:100D40006C61727320666F7220610057696C6C2051
:100D5000796F7520706179203130303000596F75AE
:100D600072206865616C74683A20007374696C6CF9
:100D700020616674657220796F7521002070696743
:100D80007300546865726520617265200042656970
:100D90006E67206368617365642121005769746818
:100DA00064726177204D6F6E6579004465706F7372
:100DB0006974204D6F6E65790042616E6B00426F01
:100DC00072726F77204D6F6E657900526570617930
:100DD000204C6F616E004C6F616E20536861726BC6
:100DE000004A65742066726F6D200053656C6C203C
:100DF0004472756773004275792044727567730099
:100E00005472656E6368636F61740042616E6B005B
:100E10004C6F616E20536861726B004A65740054B8
:100E200072656E6368636F61740053656C6C204417
:100E30007275677300427579204472756773004854
:100E40006974207468652053747265657473212118
:100E50000076312E312E3100536C616E67696E273A
:100E6000001E1E0000C08000000000000000008086
:100E70007807067880000000000000000000C040F5
:100E8000000000033CC10204081020C000FF000065
:100E90000000FF00C02010080404C2390700003819
:100EA000509090902324485060812608E70090E7F6
:100EB00008260160504826A1909090503000000014
:100EC0000000010222322A2422100A080C081221F2
:100ED000242A320203000000000000080B00020276
:100EE00002000009040000010202000005240010B5
:100EF000010524010101042402060524060001075E
:100F000005810310004009040100020A00000007E7
:100F100005020240000007058302400000040309A7
:100F20000412010002EF020140412336800001015A
:100F300002030141726475696E6F204C4C4300419D
:100F4000726475696E6F204C656F6E6172646F00BC
:100F500003051F0E0400231DC42F11241FBECFEF55
:100F6000DAE0DEBFCDBF12E0A0E0B1E0E8E4FDE6EC
:100F700002C005900D92AC36B107D9F727E0ACE678
:100F8000B2E001C01D92AC3AB207E1F717E0CCEA3B
:100F9000D7E004C02197FE010E949F34CB3AD107CD
:100FA000C9F70E94A41D0C9497360C940000EEEF34
:100FB000F2E0A0E0B8E000800EBC8111012C119796
:100FC000A0FDFDCF0192B9F70DB40895480F592F38
:100FD000511D1416150684F5803891056CF597FFA0
:100FE00002C090E080E04138510514F040E850E044
:100FF000481BFB01E770FF2721E001C0220FEA95A3
:10100000EAF777FF02C0695F7F4FFB0133E0F59598
:10101000E7953A95E1F7F695FE2FEE27F795E795D8
:10102000E80FF91FE250FD4F415030F08191DF0190
:101030001197822B8C93F8CF08956F927F928F92A5
:101040009F92AF92BF92CF92DF92EF92FF920F9357
:101050001F93CF93DF93DC01FA01149131965491E1
:101060003196C12FD0E0222309F1CC24C394D12C96
:10107000852F877011F4D12CC12CE52EE694E694CF
:10108000E694EC0CFD2CF11CEC9EC001ED9E900D45
:10109000FC9E900D1124033011F4880F991F289F96
:1010A0007001299FF00C1124EE0DFF1D7D01EC0E47
:1010B000FD1E1E141F040CF06BC0A038B1050CF00F
:1010C00067C0CB01850F911D181619060CF060C082
:1010D000603471050CF05CC0309709F459C0362FAC
:1010E0003770CB0177FD079623E0959587952A9574
:1010F000E1F7282F77FF04C0332311F02FEF280FDB
:10110000662777276A1B7B0BB7FD02C070E060E0A3
:1011100090E89A1B40E8E416F1040CF4912F961B1A
:10112000E22E022E000CFF08DE2CD0942F3F0CF094
:10113000D12C41E0852F877009F440E0B52EB6949C
:10114000B694B6944B0DE40EF11C89E0E816F10458
:1011500014F048E0421BB42EBD182D0D40E82403C6
:1011600070011124AE0DBF1DA60FB71F1D9D600D90
:10117000711D1124AF01460F571FC32E032E000C03
:10118000DD08033009F4C7C090F4023009F474C0DC
:10119000DF91CF911F910F91FF90EF90DF90CF9053
:1011A000BF90AF909F908F907F906F9008950A3F6F
:1011B000A1F1B20E0B3F61F72B1551F3BD01625047
:1011C0007D4F10E000E0091708F09FC0FA01E00F22
:1011D000F11FE491F0E04F010C2C02C0880C991C27
:1011E0000A94E2F727FD06C0FB018081F82CF094F9
:1011F0008F218083332361F0273054F47B01F0E8A2
:10120000EF0EF11CA92CA094F70180818A21808324
:101210000F5F1F4F6F5F7F4FD6CFB20E2B1509F4B4
:10122000B7CFBD0162507D4F10E000E0091708F014
:1012300066C0FA01E00FF11FE491F0E04F010C2CC1
:1012400002C0880C991C0A94E2F727FD04C0FB0138
:10125000808188298083332351F0273044F47B0137
:10126000F0E8EF0EF11CF7018081892980830F5F80
:101270001F4F6F5F7F4FDACF6FEF70E0032E02C01A
:10128000660F771F0A94E2F760957095972E8B2C66
:10129000820E281509F47CCF8D0102501D4FF12CD0
:1012A000E12CE91630F5FA01EE0DFF1DE491F0E0B6
:1012B0003F010C2C02C0660C771C0A94E2F727FD54
:1012C00005C0F8018081862386298083332359F065
:1012D00027304CF45801F0E8AF0EB11CF5018081C5
:1012E000892187298083FFEFEF1AFF0A0F5F1F4FC5
:1012F000D8CF2F5F4C0F5D1FA058BF4FCACF2F5FB5
:101300004C0F5D1FA058BF4F89CF2F5F4C0F5D1F43
:10131000A058BF4F51CFE92EF12CFA01E60FF71F6D
:10132000A250BD4F60E870E06E197F09CE19DF0949
:101330008E01000F111F41E050E07A01032E01C021
:10134000EE0C0A94EAF7592F4B2D892E932ECF934A
:10135000DF93ED01EF96EF962296A590C590992028
:1013600059F0AE9C5001CE9C600127302CF4F880DF
:10137000D094FD20FB28F99222233AF0FC90C094EF
:10138000FC20FA28FD920C94C60911965A9529F76B
:101390004A9551F0582D23951124E00FF11DA60F09
:1013A000B11DC60FD11DD9CFDF91CF911124F0CE41
:1013B0000F9302E020E00E941D080F9108952F92E4
:1013C0003F924F925F926F927F928F929F92AF92D5
:1013D000BF92CF92DF92EF92FF920F931F93CF9322
:1013E000DF93CDB7DEB728970FB6F894DEBF0FBEF8
:1013F000CDBF6F836A0119011C830B83FE82ED82CE
:10140000811128C005E010E029E030E03A8329830B
:10141000B6010D2C000C880B990B0E9403314B0177
:101420005C015F8151111DC0ECE6F7E090E080E0C7
:1014300018861F828C159D050CF02BC124813581E7
:101440004F8158854217530714F438872F8301962C
:101450003696F0CF04E010E048E050E05A8349832C
:10146000D7CF20E030E040E05FE30E9462314B01E3
:101470005C0120E030E0A9010E943D3420E030E032
:1014800040E05FE387FD30C0C501B4010E94D13266
:101490000E94AF3378876F83A6018F819885481BA0
:1014A000590BECE6F7E090E080E0B12CA12C2F8105
:1014B000388582179307ECF086E0829FF001839FC6
:1014C000F00D1124E459F84F90E080E0D12CC12CAC
:1014D00084179507BCF424813581C216D3060CF419
:1014E000690101963696F4CFC501B4010E94D0324D
:1014F000CFCF24813581A216B3060CF45901019691
:101500003696D5CFB801110F880B990B0E94033185
:101510002B013C01B5016C0D7D1D072E000C880BC5
:10152000990B0E94033120E030E040EE5FE30E941F
:10153000D1326B017C0120E030E040E05FE3C30189
:10154000B2010E9462319B01AC01C701B6010E9449
:1015500062316B017C0120E030E0A9010E943D3442
:1015600020E030E040E05FE387FD89C0C701B601BD
:101570000E94D1320E94AF3302E410E0061B170B29
:10158000F10111830083B501BB0C880B990B0E94FC
:10159000033120E030E040EE5FE30E94D132A3014E
:1015A00092010E9462314B015C0120E030E0A90110
:1015B0000E943D3420E030E040E05FE387FD64C0FE
:1015C000C501B4010E94D1320E94AF33600F711F78
:1015D000EB81FC817183608329813A81B901330FEA
:1015E000880B990B0E94033120E030E040E05FE37C
:1015F0000E9462316B017C014F815885BA01550F01
:10160000880B990B0E9403319B01AC01C701B60105
:101610000E9462316B017C0120E030E0A9010E9450
:101620003D3420E030E040E05FE387FD85C0C70146
:10163000B6010E94D1320E94AF332AE230E0C901E4
:10164000861B970BED81FE819183808328960FB6D0
:10165000F894DEBF0FBECDBFDF91CF911F910F91E8
:10166000FF90EF90DF90CF90BF90AF909F908F90C2
:101670007F906F905F904F903F902F900895C7019B
:10168000B6010E94D03276CFC501B4010E94D0329B
:101690009BCFB801110F880B990B0E94033120E0FA
:1016A00030E040E05FE30E9462312B013C01EF81BA
:1016B000F885BF01FF0F880B990B0E9403319B0136
:1016C000AC01C301B2010E9462312B013C0120E058
:1016D00030E0A9010E943D3420E030E040E05FE3CB
:1016E00087FD25C0C301B2010E94D1320E94AF33F1
:1016F00022E430E0C901861B970BF10191838083BE
:101700008FEF9FEFEB81FC819183808329813A8168
:10171000B901330F880B990B0E94033120E030E0B0
:1017200040E05FE30E946231A501940171CFC301E3
:10173000B2010E94D032DACFC701B6010E94D03286
:101740007ACFFC018091FD02882311F13FB7F89414
:1017500082E08093E9002091F200822F90E0181639
:10176000190614F481E090E0882339F0289844E6C3
:101770004093FC024091F1004083222339F02091F4
:10178000F200211103C02BE62093E8003FBF08952B
:101790008FEF9FEF08952FB7F89483E08093E900CF
:1017A0009091E800892F807295FF04C09091F2001B
:1017B00080E4891B2FBF08958091F40281110DC030
:1017C00082E08093F00284E08093F1021092F302B1
:1017D0001092F20281E08093F40280EF92E008958B
:1017E000CF93DF931F92CDB7DEB76983DC01ED9114
:1017F000FC910280F381E02D41E050E0BE016F5F7B
:101800007F4F09950F90DF91CF91089583E08093EA
:10181000E9008091F200882319F08AE38093E800C0
:1018200008950E94CB0B90E00895CF93DF931F9211
:10183000CDB7DEB7FC018485958597FD08C02FEFF5
:101840003FEF358724870F90DF91CF910895CE0128
:1018500001960E94A10B019719F4898190E0F3CFC2
:101860008FEF9FEFF0CF0F931F93CF93DF931F92D4
:10187000CDB7DEB78C01FC018485958597FF0BC041
:10188000CE0101960E94A10B019771F4898190E02D
:10189000F80195878487F801848595850F90DF91FD
:1018A000CF911F910F9108958FEF9FEFF1CFFC0122
:1018B0008485958597FD0BC09FB7F89482E080934F
:1018C000E9008091F2009FBF90E0019608959FB7D4
:1018D000F89482E08093E9008091F2009FBF90E04D
:1018E00008954091EA025091EB022091E802309174
:1018F000E90242175307B4F49091E8009570E1F3C0
:101900009091E80092FD19C08093F1008091EA0265
:101910009091EB0201968F739927892B19F48EEF22
:101920008093E8008091EA029091EB0201969093F7
:10193000EB028093EA0281E0089580E00895DF924F
:10194000EF92FF920F931F93CF93DF93D82E8A01CC
:10195000EB017B01E40EF51ECE15DF0559F0D7FE35
:1019600012C0FE0184910E94710C21968111F4CF66
:101970000FEF1FEFC801DF91CF911F910F91FF90E3
:10198000EF90DF9008958881EECF0F931F93CF9350
:10199000DF931F92CDB7DEB782E0898342E450E047
:1019A0006BED7EE080E80E949F0C0E94DC0BDC0166
:1019B00012960D911C910115110589F0D801ED9138
:1019C000FC910280F381E02DBE016F5F7F4FC80163
:1019D000099597FD04C0F80100851185ECCF898138
:1019E0000F90DF91CF911F910F910895615030F0CA
:1019F0002091F100FC0120830196F8CF289884E61D
:101A00008093FC0208953FB7F8948091E40290918E
:101A1000E502A091E602B091E70226B5A89B05C0B9
:101A20002F3F19F00196A11DB11D3FBFBA2FA92F5D
:101A3000982F8827BC01CD01620F711D811D911D5A
:101A400042E0660F771F881F991F4A95D1F70895C6
:101A50008F929F92AF92BF92CF92DF92EF92FF92BE
:101A60006B017C010E94030D4B015C01C114D10488
:101A7000E104F104B9F00E94030D681979098A099B
:101A80009B09683E73408105910580F321E0C21AED
:101A9000D108E108F10888EE880E83E0981EA11CA9
:101AA000B11CE4CFFF90EF90DF90CF90BF90AF904C
:101AB0009F908F9008958F929F92AF92BF92CF92F6
:101AC000DF92EF92FF920F931F93CF93DF936C01FE
:101AD0007B018A0180910C01882309F45CC080910C
:101AE000FD02882309F457C08091EF0280FF05C0F2
:101AF0008091E00082608093E000E801B12C8AEFE1
:101B0000A82E93E0892E2AE3922E209711F4BB2071
:101B1000D9F10E94CB0B81110AC0AA94AA20D9F155
:101B200061E070E080E090E00E94280DEECF8C171D
:101B30001D0611F00CF08C2F9FB7F8948092E900ED
:101B40002091E80025FD02C09FBFDFCF282F30E0A5
:101B5000C21BD30BF701815020F041914093F1005B
:101B6000FACFE20EF31EBB2021F09092E800B12CD8
:101B7000EBCF8091E80085FDE7CF9092E800BB2491
:101B8000B394209709F3F3CF5D9884E68093EE0237
:101B9000101611063CF081E090E0F60193838283F9
:101BA00010E000E0C801DF91CF911F910F91FF90ED
:101BB000EF90DF90CF90BF90AF909F908F9008955F
:101BC0000895DB0114964D915C9115976D917C9170
:101BD000DC01ED91FC910280F381E02D09942F92BC
:101BE0003F924F925F926F927F928F929F92AF92AD
:101BF000BF92CF92DF92EF92FF920F931F93CF93FA
:101C0000DF9300D000D000D0CDB7DEB7782E662E9F
:101C10005A0128E0422E512C811103C099E0492E2F
:101C2000512CCE0101967C018E010D5F1F4F9E014C
:101C30002B5F3F4FA501662D872D0E94DF09B5015F
:101C40000B2C000C880B990B0E94033120E030E034
:101C500040E05FE30E9462316B017C0120E030E0F4
:101C6000A9010E943D3420E030E040E05FE387FDC1
:101C700024C0C701B6010E94D1320E94AF338B014C
:101C80008CE6C82E87E0D82E049D1001059D300CEF
:101C9000149D300C1124F12CE12C912C812C8A14F0
:101CA0009B04B4F589819A81662019F0801691060B
:101CB0004CF42D818E0D9F1D0BC0C701B6010E94F3
:101CC000D032DBCF2B81A70142195309840F951F16
:101CD0007720A1F02093950720939407809396078F
:101CE000B60180E997E00E94E10D9FEF891A990AF9
:101CF00086E0C80ED11CE40CF51CD1CF20939F07C1
:101D000020939E078093A007B6018AE997E0EBCF66
:101D100026960FB6F894DEBF0FBECDBFDF91CF91F0
:101D20001F910F91FF90EF90DF90CF90BF90AF90F9
:101D30009F908F907F906F905F904F903F902F90EB
:101D40000895EF92FF920F931F93CF93DF938C012F
:101D50007B01D0E0C0E0F701EC0FFD1F649166232A
:101D600061F0D801ED91FC910190F081E02DC80166
:101D70000995892B11F02196EECFCE01DF91CF91FD
:101D80001F910F91FF90EF900895AF92BF92CF9265
:101D9000DF92EF92FF920F931F93CF93DF936C012B
:101DA0007B018B01040F151FEB015E01AE18BF080C
:101DB000C017D10759F06991D601ED91FC910190BE
:101DC000F081E02DC6010995892B79F7C501DF91D6
:101DD000CF911F910F91FF90EF90DF90CF90BF9028
:101DE000AF9008952D9A0895BC0190E080E00C9486
:101DF000280D8FB18095807F669B88601C9B8460D6
:101E0000089581EC80937C0085B1806F85B984B1A1
:101E1000877E84B984B1876E84B95E9A5F988AB1EF
:101E2000806D8AB9769A6E9881B3806F81BB8998EC
:101E300080B38D7080BB80E58CBD81E08DBD85E079
:101E400090E00E94F40E5F9A85E090E00E94F40E0C
:101E50005E985C98ECE1F8E084918EBD00000DB4D2
:101E600007FEFDCF319688E0E932F807A9F75C9AC2
:101E700081E88093640080916500816080936500B3
:101E8000089590917402982329F4909175029823F3
:101E900081E009F480E00895CF93C82F0E94F90EE5
:101EA000982F9C2381E09C1380E0CF91089580E0DF
:101EB0000C94D70780389105B8F460347105A0F40C
:101EC00020E191E061FD94E060FD990F62FD929543
:101ED000687F269FD0011124A80FA250BD4F8C917E
:101EE00040FF03C0892B8C93089590958923FBCFE5
:101EF0002F923F924F925F926F927F928F929F921A
:101F0000AF92BF92CF92DF92EF92FF920F931F9307
:101F1000CF93DF937C016B0188248394912CD0E0D4
:101F2000C0E005E010E096EF692E77247A942CEF5C
:101F3000A22EBB24BA94842F8470582E842F8270D2
:101F4000482E842F8870382E4170242E219682E0EE
:101F5000880E911CA80CB91C552091F041E0B801E5
:101F60006C0D7D1DC7018C0F9D1F0E945A0F41E013
:101F7000B6016C0F7D1FC8018E0D9F1D0E945A0F68
:101F8000442091F041E0B601601B710BC7018C0F3A
:101F90009D1F0E945A0F41E0B6016C1B7D0BC801CA
:101FA0008E0D9F1D0E945A0F332091F041E0B60123
:101FB0006C0F7D1FC701801B910B0E945A0F41E0DF
:101FC000B8016C0D7D1DC7018C1B9D0B0E945A0F23
:101FD000222091F041E0B6016C1B7D0BC701801BF4
:101FE000910B0E945A0F41E0B601601B710BC701B3
:101FF0008C1B9D0B0E945A0FC017D10754F4B7FCDD
:10200000A5CF0150110982E0680E711CA60CB71C07
:102010009DCFDF91CF911F910F91FF90EF90DF90B7
:10202000CF90BF90AF909F908F907F906F905F9078
:102030004F903F902F9008952F923F924F925F9232
:102040006F927F928F929F92AF92BF92CF92DF92C8
:10205000EF92FF920F931F93CF93DF93EC0141E038
:102060006FE370E00E945A0F41E065E370E0CE013B
:102070000E945A0F41E06AE370E0CE0105960E948B
:102080005A0F41E06AE370E0CE0105970E945A0FB3
:1020900022242394312CF12CE12C05E010E036EFC2
:1020A000432E55245A944CEFC42EDD24DA948FEF3E
:1020B000E81AF80A82E0280E311CC20CD31C470132
:1020C0008C0E9D1E41E058018AE3A80EB11CB5019B
:1020D000C4010E945A0F3E016E187F0841E0B5010D
:1020E000C3010E945A0F41E08AE3A82EB12CA01A26
:1020F000B10AB501C4010E945A0F41E0B501C30104
:102100000E945A0F47018AE3880E911C41E0B401F6
:102110005E01A00EB11EC5010E945A0F41E0B4013C
:102120003E01601A710AC3010E945A0F9AE3892E78
:10213000912C8E189F0841E0B401C5010E945A0FEE
:1021400041E0B401C3010E945A0FE016F1069CF071
:10215000DF91CF911F910F91FF90EF90DF90CF9083
:10216000BF90AF909F908F907F906F905F904F90B7
:102170003F902F900895D7FC9ACF0150110982E02B
:10218000480E511CC40CD51C92CF8F929F92AF92D7
:10219000BF92CF92DF92EF92FF920F931F93CF9354
:1021A000DF936D3089F0C0907202D09073026A3074
:1021B000D1F4109271021092700288E0C80ED11C06
:1021C000D0927302C092720281E090E0DF91CF91D1
:1021D0001F910F91FF90EF90DF90CF90BF90AF9045
:1021E0009F908F9008950091700210917102E5E028
:1021F0006E9FE0011124C45EDC4F4801F12CF5E034
:10220000E12CFF1629F0CE010196FE01E490EC01CD
:10221000B12CA12C4E2D4170B6016A0D7B1DC4015D
:102220000E945A0FE694FFEFAF1ABF0A88E0A81683
:10223000B10481F7F394EFEF8E1A9E0AF6E0FF12D5
:10224000DECF0A5F1F4F1093710200937002BCCF64
:10225000DF92EF92FF920F931F93CF93DF937C0156
:10226000D22E8B01040F111DEB0177FF02C0D0E0CD
:10227000C0E0C8010134110514F080E490E0C817F3
:10228000D9073CF44D2DBE01C7010E945A0F21967B
:10229000F0CFDF91CF911F910F91FF90EF90DF90E2
:1022A00008952F923F924F925F926F927F928F92FA
:1022B0009F92AF92BF92CF92DF92EF92FF920F93D5
:1022C0001F93CF93DF9300D000D000D0CDB7DEB7FF
:1022D0006C01762E542E4901602E98E0A92EB12C67
:1022E000611103C089E0A82EB12CCE0101967C01BA
:1022F0008E010D5F1F4F9E012B5F3F4FA401652D87
:10230000872D0E94DF0909811A81552011F1B4013E
:10231000990C880B990B0E94033120E030E040E0DB
:102320005FE30E9462311B012C0120E030E0A90133
:102330000E943D3420E030E040E05FE387FD0CC0C8
:10234000C201B1010E94D1320E94AF33C616D70636
:1023500044F48D809E8009C0C201B1010E94D03238
:10236000F3CF8B809C80C61AD70ACA9CB001CB9C45
:10237000700DDA9C700D1124060F171FC40104970D
:102380006620B1F061E070E0711002C062E070E0C0
:10239000060F171F6C01C6012FEFC21AD20AC8140C
:1023A000D90491F020E045E0B8010E942811F3CF54
:1023B00061E070E0711002C062E070E0600F711FB8
:1023C00040E55FE00E94D80926960FB6F894DEBF7C
:1023D0000FBECDBFDF91CF911F910F91FF90EF9076
:1023E000DF90CF90BF90AF909F908F907F906F9035
:1023F0005F904F903F902F9008950F93CF93DF936E
:10240000EC019E816A3059F48D818C836985960F29
:102410009E8381E090E0DF91CF910F910895262F68
:1024200061E0690F2A3398F4203378F5273249F1B7
:1024300040F4213261F198859C5F8C81890F8C83F7
:10244000E8CF2C3231F12E32B1F72FE309C021341D
:1024500090F32B35C0F08FE9820F27548A3158F75B
:10246000062E000C770B8C81082E000C990B3F81F7
:102470000AEF313009F00BEF42E152E00E941D08F3
:10248000DACF21E4EDCF2154EBCF2C5FE9CF2EE35F
:10249000E7CF20E4E5CF0F93CF93DF93EC019E814C
:1024A0006A3059F48D818C836985960F9E8381E013
:1024B00090E0DF91CF910F910895262F61E0690F91
:1024C0002A3398F4203378F5273249F140F4213249
:1024D00061F198859D5F8C81890F8C83E8CF2C32C8
:1024E00031F12E32B1F72FE309C0213490F32B35AF
:1024F000C0F08FE9820F27548A3158F7062E000C5E
:10250000770B8C81082E000C990B3F810AEF31303C
:1025100009F00BEF4AE451E00E941D08DACF21E4F4
:10252000EDCF2154EBCF2C5FE9CF2EE3E7CF20E4B2
:10253000E5CFE8EBF2E080ED92E030E020E0419181
:10254000519161917191240F351F8E179F07B9F733
:102550008091850290918602821B930B0895E091F1
:10256000D802F091D9023297E531F10508F034C074
:10257000E454FD4E0C949F34D712EC12D412DA12AC
:10258000DD12EC12EC12D112E012EC12EC12EC1291
:10259000EC12EC12EC12E712E712EC12D412EC126D
:1025A000D41282E090E0089581E090E0089583E005
:1025B00090E0089584E090E0089585E090E008952B
:1025C00080919702909198020397029728F4809146
:1025D000950290919602089590E080E00895CF933F
:1025E000C82F84E00E94410F811107C0CC23B1F0B5
:1025F00088E00E94410F882389F01092DE020E9439
:10260000AF129093DD028093DC028091970290914B
:1026100098029093D9028093D80281E0CF910895D7
:10262000E0E9F7E08AE48583848387E3868368EDC5
:1026300070E0CF010E94A10E8BE490E00E941C107C
:1026400087E690E00C941C10CF92DF92EF92FF92FD
:102650000F931F93CF93DF9346E770E060E085E030
:1026600090E00E94E60746E76FE370E085E090E0C7
:102670000E94E60721E046E365E070E090E080E03C
:102680000E94281121E046E365E070E08FE790E0CA
:102690000E94281141E065E070E085E090E00E9432
:1026A000780F42E065E070E08AE790E00E94780FE2
:1026B00044E06AE370E08AE790E00E94780F48E027
:1026C0006AE370E085E090E00E94780F80919902C3
:1026D000CEE4D7E0811122C00AE010E0F12CE12C19
:1026E0008AE0C82ED12C80919A0290919B02E81624
:1026F000F90684F58FEFE81AF80AD0927102C092B9
:1027000070021093730200937202BE0184EA97E094
:102710000E94E10D065F1F4F2696E5CF1AE0F12CCF
:10272000E12C0AE080919A0290919B02E816F9064A
:102730008CF400939F0700939E071093A007BE019F
:102740008AE997E00E94E10D8FEFE81AF80A175F17
:102750002696E8CFDF91CF911F910F91FF90EF90D8
:10276000DF90CF900895BC01EAE9F7E096E0958309
:1027700094838CE08683CF010C94E10D90E080E09F
:1027800008958F929F92AF92BF92EF92FF920F9314
:102790001F93CF93DF93CDB7DEB7A1970FB6F89411
:1027A000DEBF0FBECDBF7C01FA01CB0119A22230E2
:1027B00008F42AE08E010F5D1F4F822E912CB12C60
:1027C000A12CBF01A50194010E949F32F901CA0109
:1027D0006A3074F5605DD8016E938D01232B242B34
:1027E000252B79F790E080E0109789F0FD010190AA
:1027F0000020E9F73197AF014A1B5B0BD701ED9140
:10280000FC910280F381E02DB801C7010995A196E2
:102810000FB6F894DEBF0FBECDBFDF91CF911F91F1
:102820000F91FF90EF90BF90AF909F908F90089581
:10283000695CD1CFCF92DF92EF92FF920F931F93FB
:10284000CF93DF9377FF21C06A017B01EC01E88120
:10285000F9810190F081E02D6DE209958C0144270A
:102860005527BA014C195D096E097F092AE0CE018E
:102870000E94C113800F911FDF91CF911F910F9183
:10288000FF90EF90DF90CF9008952AE0DF91CF91F5
:102890001F910F91FF90EF90DF90CF900C94C11398
:1028A000CF93DF93CFE1D0E020E04AE067E170E032
:1028B000CE010E9428112196CF36D105A9F783E2D7
:1028C00080939F0780939E0788E18093A0074091A3
:1028D00081025091820260918302709184028AE9A0
:1028E00097E0DF91CF910C941A14BC01EAE9F7E06C
:1028F0009AE09583948388E18683CF010E94E10D5D
:1029000048E566E170E08EE190E00E94E60748E568
:1029100061E270E08EE190E00E94E60721E04CE089
:1029200066E170E08EE190E00E94281121E04CE029
:1029300066E170E085E790E00E9428110E94501443
:1029400041ED50E068E170E08FE690E00C94D8092A
:10295000CF92DF92EF92FF920F931F93CF93C82FE6
:102960008B0169017A016E5F7F4F4AEC50E00E9453
:10297000D809CA5FEAE9F7E0C583C4830683B701D3
:10298000A601CF01CF911F910F91FF90EF90DF90A3
:10299000CF900C941A14CF93DF938091D80290912A
:1029A000D9024197029768F5C8E2D0E020E047E0FD
:1029B00065E270E0CE010E9428112196CF37D10543
:1029C000A9F7E0919502F0919602EE0FFF1FEE0F2E
:1029D000FF1FE056FD4F208131814281538160917C
:1029E00081027091820280918302909184020E9400
:1029F0008F349B01AC0165E270E088E290E00E94B8
:102A0000A814DF91CF910C945014CF93DF93EC0175
:102A100088819981009711F00E94413519821882AE
:102A20001D821C821B821A82DF91CF910895FC01C6
:102A300080819181009711F00C9441350895CF93D6
:102A4000C82F8091D6029091D70201969093D70219
:102A50008093D602109280020E94333021EE3EE233
:102A600040E050E00E9436326058714C8F4F9F4FCB
:102A70006093A0027093A1028093A2029093A3029C
:102A80000E94333029E53BE140E050E00E943632BD
:102A900068577C4E8F4F9F4F6093A4027093A5029E
:102AA0008093A6029093A7020E94333023E230E085
:102AB00040E050E00E9436329B01AC01265F3F4F60
:102AC0004F4F5F4FA4E6B0E00E9455326093A802DA
:102AD0007093A9028093AA029093AB020E943330B4
:102AE0002BE230E040E050E00E9436329B01AC0126
:102AF0002F5D3F4F4F4F5F4FAAE0B0E00E9455322D
:102B00006093AC027093AD028093AE029093AF02DB
:102B10000E94333020E130E040E050E00E94363245
:102B20009B01AC01295F3F4F4F4F5F4FAAE0B0E0E0
:102B30000E9455326093B0027093B1028093B2024A
:102B40009093B3020E94333025E030E040E050E043
:102B50000E9436329B01AC012F5F3F4F4F4F5F4FBA
:102B6000AAE0B0E00E9455326093B4027093B502BF
:102B70008093B6029093B702CC23C1F160918D028D
:102B800070918E0280918F02909190020E94033189
:102B90002DEC3CEC4CE85FE30E9462310E94E5338F
:102BA0000E94AF3360938D0270938E0280938F02E8
:102BB000909390026091890270918A0280918B02B9
:102BC00090918C020E94033124E13EEA47E85FE3E2
:102BD0000E9462310E94E5330E94AF336093890204
:102BE00070938A0280938B0290938C021092DE0283
:102BF000CF9108950C9420320F931F93CF93DF93BE
:102C00008C01EB01FC01808191810097E1F06881EA
:102C1000798161157105A9F0428153812C813D8133
:102C20004217530770F00E9490368C819D81F80105
:102C3000958384831D821C82DF91CF911F910F9118
:102C400008950E94413588819981F801918380839C
:102C50008A819B81938382838C819D8195838483E8
:102C6000198218821B821A82E5CF0F931F93CF938C
:102C7000DF93EC0188819981009759F02A813B818B
:102C80002617370730F081E0DF91CF911F910F9128
:102C900008958B016F5F7F4F0E94CA35009759F0EE
:102CA000998388831B830A832C813D81232B59F7C9
:102CB000FC011082E8CF80E0E7CFEF92FF920F9304
:102CC0001F93CF93DF93EC017B01CB010E949230E5
:102CD0000097A9F00C811D81080F191FB801CE01C2
:102CE0000E943516882361F0288139818C819D816D
:102CF000B701820F931F0E948B301D830C8381E0EC
:102D0000DF91CF911F910F91FF90EF900895EF9277
:102D1000FF920F931F93CF93DF93FB01E080F1802D
:102D2000E114F10441F480E0DF91CF911F910F9104
:102D3000FF90EF9008950481158101151105B1F000
:102D4000EC018C819D81080F191FB801CE010E94F2
:102D50003516882341F3288139818C819D81B70103
:102D6000820F931F0E9490361D830C8381E0DCCF7D
:102D7000EF92FF920F931F93CF93DF93EC018B01A0
:102D80006115710551F0CB010E9492307C01BC01AC
:102D9000CE010E94351681110BC0CE010E9405158F
:102DA000CE01DF91CF911F910F91FF90EF90089589
:102DB000FD82EC82B801888199810E948B30F0CF2E
:102DC000FC011182108213821282158214820C94EB
:102DD000B816CF93DF93EC016230710501F148F42E
:102DE0006115710581F061307105B1F06FE171E03D
:102DF0000CC064307105C9F0A8F065307105B1F7F9
:102E000060E271E002C06EE371E0CE010E94E01664
:102E1000CE01DF91CF91089566E371E0F6CF61E3D3
:102E200071E0F3CF6CE271E0F0CF66E271E0EDCFDC
:102E3000CF93DF93EC016230710501F148F4611525
:102E4000710581F061307105B1F064EE70E00CC085
:102E500064307105C9F0A8F065307105B1F765EE11
:102E600070E002C069E171E0CE010E94E016CE017F
:102E7000DF91CF91089562E171E0F6CF65E071E0F6
:102E8000F3CF6BEF70E0F0CF6EEE70E0EDCFEF922E
:102E9000FF920F931F93CF93DF93EC017B018A0185
:102EA000BA010E94351681110BC0CE010E94051592
:102EB000CE01DF91CF911F910F91FF90EF90089578
:102EC0001D830C83B701888199810E949036F0CFD1
:102ED000FB0101900020E9F73197AF01461B570B2A
:102EE0000C9447170F931F93CF93DF93CDB7DEB7A3
:102EF00062970FB6F894DEBF0FBECDBF8C01CB0139
:102F0000F8011182108213821282158214824AE023
:102F1000BE016F5F7F4F0E949B30BE016F5F7F4F8E
:102F2000C8010E94681762960FB6F894DEBF0FBE04
:102F3000CDBFDF91CF911F910F9108950F931F93F4
:102F4000CF93DF93CDB7DEB7A2970FB6F894DEBF6D
:102F50000FBECDBF8C01CB01BA01F80111821082E6
:102F600013821282158214822AE0AE014F5F5F4FF6
:102F70000E94A630BE016F5F7F4FC8010E94681794
:102F8000A2960FB6F894DEBF0FBECDBFDF91CF91F2
:102F90001F910F9108952F923F924F925F926F92DF
:102FA0007F928F929F92AF92BF92CF92DF92EF92D9
:102FB000FF920F931F93CF93DF93CDB7DEB7629746
:102FC0000FB6F894DEBF0FBECDBF2C019E012F5F60
:102FD0003F4F490139011C01D12CC12C10E000E008
:102FE000B12CA12CF10141915191619171911F017D
:102FF000CE010D960E949E17E988FA88CE010D96A3
:103000000E941715B601CE010D960E94E916898916
:103010009A89E80EF91EFFEFEF1AFF0AF301E19219
:10302000F1923F01CE010D960E941715F3E0CF16E5
:10303000D1040CF03FC0AE14BF040CF457012FEFC5
:10304000C21AD20A36E0C316D10461F68CE6C82E45
:1030500087E0D82EF12CE12C150183E0E816F1046D
:103060000CF01801B701CE010D960E94E916BE01C1
:10307000635F7F4FC6010E94FC15CE010D960E9432
:10308000171568E471E0C6010E945D16712C612C71
:10309000F401808191819101281B390B621673061E
:1030A00074F466E471E0C6010E945D163FEF631A96
:1030B000730AEECF0E151F0514F68701C0CFF2017B
:1030C00041915191619171912F01CE010D960E9414
:1030D0009E17BE01635F7F4FC6010E948716CE0117
:1030E0000D960E941715FFEFEF1AFF0A26E0C20E99
:1030F000D11C32E0830E911C86E0E816F10409F041
:10310000ABCFF092D502E092D40281E08093D2025C
:103110000A0D1B1D073111050CF480E08093D302CA
:1031200062960FB6F894DEBF0FBECDBFDF91CF9190
:103130001F910F91FF90EF90DF90CF90BF90AF90D5
:103140009F908F907F906F905F904F903F902F90C7
:103150000895EF92FF920F931F93CF93DF9300D0C8
:1031600000D000D0CDB7DEB78C019CE3E92EF12C66
:1031700020E04CE069E070E0C7010E9428118FEF69
:10318000E81AF80A80E8E816F10491F7000F111F19
:10319000000F111FF801E854FD4F408151816281F9
:1031A0007381CE0101960E949E178D818195880FB3
:1031B000880F845A80939507809394078DE08093BD
:1031C000960748E050E064E571E080E997E00E94EE
:1031D000C50EBE016F5F7F4F80E997E00E94E10D51
:1031E000CE0101960E94171526960FB6F894DEBF01
:1031F0000FBECDBFDF91CF911F910F91FF90EF9048
:103200000895EF92FF920F931F93CF93DF9300D017
:1032100000D000D0CDB7DEB78091D8029091D9020E
:10322000099709F05EC00E9499128C01BC01CE0181
:1032300001960E947217ED80FE80CE0101960E94D9
:10324000171581E080939507809394071092960755
:1032500064EC70E080E997E00E94A10E4091870243
:1032600050918802052E000C660B770B80E997E0E1
:103270000E941A1487E190E08E199F09880F991F08
:10328000880F991F80939507809394071092960753
:103290006AEB70E080E997E00E94A10EA801110F8F
:1032A000660B770B80E997E00E941A1410E000E0AB
:1032B00021E041E068E070E0C8010E9428110F5F42
:1032C0001F4F00381105A1F726960FB6F894DEBF00
:1032D0000FBECDBFDF91CF911F910F91FF90EF9067
:1032E00008954091910250919202609193027091E1
:1032F0009402CE0101960E949E17ED80FE80CE01C1
:1033000001960E94171500E210E00E191F09000F28
:10331000111F000F111F8091D8029091D9029C01BA
:10332000255031092230310508F052C021E02093A8
:103330009507209394071092960760EB70E005972D
:1033400011F465EB70E080E997E00E94A10E4AEC71
:1033500050E061E070E083E190E00E94D80989E1EB
:103360008093950780939407109296078091D802D6
:103370009091D902059719F540918D0250918E02D6
:1033800060918F027091900280E997E00E941A1478
:103390004AEC50E061E070E0C80106970E94D8094D
:1033A000009395070093940710929607409191021D
:1033B00050919202609193027091940273CF409168
:1033C000890250918A0260918B0270918C02DCCF4D
:1033D00081E08093950780939407109296076CEA9A
:1033E00070E080E997E00E94A10E8EE0809395073F
:1033F00080939407109296074091D6025091D7027D
:10340000052E000C660B770BBFCF1F920F920FB6E5
:103410000F9211248F939F938091E1009091E1008E
:10342000937F9093E10083FF0FC01092E90091E039
:103430009093EB001092EC0092E39093ED001092C9
:10344000FD0298E09093F00082FF22C093E09093F9
:10345000E9009091F200992319F09AE39093E80023
:103460009091EE02992341F09091EE029150909349
:10347000EE02911101C05D9A9091FC02992341F0F6
:103480009091FC0291509093FC02911101C0289AF6
:1034900084FF18C08091E2008E7E81608093E200FC
:1034A0008091E1008F7E8093E1008091EF028E7E1B
:1034B00080618093EF029F918F910F900FBE0F90CC
:1034C0001F90189580FFF7CF8091E2008E7E80617B
:1034D0008093E2008091E1008E7E8093E1008091F4
:1034E000EF028E7E8160E5CF1F920F920FB60F9292
:1034F0001124CF92DF92EF92FF920F931F932F939D
:103500003F934F935F936F937F938F939F93AF936B
:10351000BF93EF93FF93CF93DF93CDB7DEB76C9755
:10352000DEBFCDBF1092E9008091E80083FF25C087
:1035300068E0CE0145960E94F60C82EF8093E80089
:103540008D8987FF39C09091E80090FFFCCF982FBC
:10355000907609F034C19E894F89588D2F89F88C57
:10356000911131C0803861F58091ED028093F100B6
:103570001092F1008EEF8093E8006C960FB6F894ED
:10358000DEBF0FBECDBFDF91CF91FF91EF91BF9115
:10359000AF919F918F917F916F915F914F913F91EB
:1035A0002F911F910F91FF90EF90DF90CF900F9090
:1035B0000FBE0F901F9018959EEF9093E800C7CF15
:1035C0001092F100D5CF913059F48111D3CF413011
:1035D000510581F68091ED028D7F8093ED02CACF77
:1035E000933049F48111C6CF4130510519F68091CD
:1035F000ED028260F2CF953041F48091E80080FFC7
:10360000FCCF20682093E300B5CF963009F0A9C025
:103610000B8D1C8D22E01092E9001092EB021092AB
:10362000EA02F2122EC01092E9021092E8020E9401
:10363000C50C1F8299E09983FA8291E09E8390EAFB
:1036400098879AEF99872091EA023091EB02275FE1
:103650003F4F3C832B838D831092E9001092EB0245
:103660001092EA021093E9020093E80249E050E068
:10367000BE016F5F7F4F80E00E949F0C0E94C50CCF
:1036800079CF1093E9020093E8020E94DC0BDC0181
:1036900012960D911C910115110509F451C1D80123
:1036A000ED91FC910480F581E02DBE016B5E7F4FB2
:1036B000C8010995009709F03EC1F8010085118500
:1036C000EACFF3E0FF120EC08F89882309F440C0CF
:1036D000823061F440E860E18FE39FE00E94F01CDB
:1036E000811148CF81E28093EB0047CF813029F4EC
:1036F00040E86BE083E39FE0F1CF833099F70E94CD
:10370000DC0BDC011296ED90FC908E010F5F1F4FD9
:103710006801E114F10479F0D701ED91FC91068084
:10372000F781E02DB801C7010995080F111DF701B8
:10373000E084F184EECFD8011C92F60101900020C4
:10374000E9F73197BF016C197D0940E0C601C6CF8A
:103750006DE17FE0FB01449150E080E80E949F0C06
:1037600009CF973009F4BECF983021F481E08093DF
:10377000F10000CF993009F0FDCE837009F0B2CF8F
:10378000E8E1F1E081E031E096E32191222371F05C
:103790008093E9003093EB00DF0111972C91209387
:1037A000EC009093ED008F5F873079F78EE7809380
:1037B000EA001092EA008F898093FD02DBCE8B8DA8
:1037C0009C8D1092E9001092EB021092EA02909305
:1037D000E9028093E802898D811192C08E899D89CA
:1037E000913A49F4813209F07DCF47E050E065E03D
:1037F00071E080E0B3CF913209F074CF833269F485
:103800008F89988DB0E0A0E0809301019093020130
:10381000A0930301B0930401ADCE803269F480918E
:10382000E80082FFFCCF67E085E091E00E94F60CA3
:103830008BEF8093E8009ECE823209F09BCE8F8979
:1038400080930C01EEEFFFE7859194918B3F9C4DA7
:1038500051F1E0E0F8E08091050190910601A0911E
:103860000701B0910801803B9440A105B105F1F436
:1038700080910C0180FD1AC0EE3F8AE0F80789F5BF
:1038800087E797E791838083809160008093EC02C3
:1038900088E19BE00FB6F894A895809360000FBE76
:1038A0009093600067CEEEEFFAE0D5CF80819181F2
:1038B0008737974709F05ECEA895809160008861B0
:1038C000809360008091EC0280936000EE3F2AE0DC
:1038D000F20789F08091FE0A9091FF0A918380831C
:1038E00049CE808191818737980751F29093FF0AE2
:1038F0008093FE0AC5CF1092FF0A1092FE0A3ACEBC
:103900000E94DC0BDC0112960D911C910115110532
:1039100009F4E8CED801ED91FC910190F081E02D01
:10392000BE016B5E7F4FC8010995811123CEF8015E
:1039300000851185EBCF181619060CF41BCED2CEDC
:10394000F1E0FF12BECE61E27FE004CF1F920F9242
:103950000FB60F9211242F933F938F939F93AF93A2
:10396000BF938091E0029091E102A091E202B091B8
:10397000E3023091DF0223E0230F2D3758F5019643
:10398000A11DB11D2093DF028093E0029093E1021C
:10399000A093E202B093E3028091E4029091E502E9
:1039A000A091E602B091E7020196A11DB11D80939E
:1039B000E4029093E502A093E602B093E702BF9180
:1039C000AF919F918F913F912F910F900FBE0F90CC
:1039D0001F90189526E8230F0296A11DB11DD2CF86
:1039E000EF92FF920F931F93CF93DF93F82E192F2F
:1039F000E62E042F81E0860F880F0E94710C83E071
:103A00000E94710CCF2DD12FEC0EFD2EF11CCE1586
:103A1000DF05B9F007FF13C0FE0184910E94710C0D
:103A2000182F80E00E94710C812321968111EFCF25
:103A3000DF91CF911F910F91FF90EF9008958881B2
:103A4000EDCF81E0F5CFCF93DF9310920107109275
:103A5000000788EE93E0A0E0B0E080930207909327
:103A60000307A0930407B093050782E291E09093C7
:103A7000FF068093FE068FEF9FEF90930B078093D6
:103A80000A071092A7071092A6078CE491E0909382
:103A9000A5078093A40710929D0710929C0780E4CD
:103AA00091E090939B0780939A0798E09093A307E7
:103AB00081E08093A20710929F071092A0071092B6
:103AC0009E078093A107109293071092920724E318
:103AD00031E030939107209390079093990780935A
:103AE000980710929507109296071092940780936A
:103AF0009707CCE6D7E0198218821B821A821D82B2
:103B00001C8250E040E063E072E0CE010E94471763
:103B1000269687E0C039D80771F7CEE4D7E019823E
:103B200018821B821A821D821C8250E040E063E0F2
:103B300072E0CE010E944717269687E0CC36D80760
:103B400071F7DF91CF910895CF93DF93CDB7DEB7B3
:103B50002E970FB6F894DEBF0FBECDBF789484B514
:103B6000826084BD84B5816084BD85B5826085BD79
:103B700085B5816085BD80916E00816080936E0007
:103B800010928100809181008260809381008091F9
:103B900081008160809381008091800081608093AA
:103BA00080008091910082608093910080919100CB
:103BB000816080939100809190008160809390005B
:103BC0008091C10084608093C1008091C1008260B7
:103BD0008093C1008091C10081608093C100809179
:103BE000C30081608093C3008091C0008260809395
:103BF000C0008091C20081608093C20080917A00F1
:103C0000846080937A0080917A00826080937A0049
:103C100080917A00816080937A0080917A00806838
:103C200080937A001092FD021092ED021092EF0242
:103C30008091D70081608093D70080EA8093D8007C
:103C400089B5806189BD89B5826089BD09B400FEEE
:103C5000FDCF61E070E080E090E00E94280D80914F
:103C6000D8008F7C80618093D8008091E000807FB5
:103C70008093E0008091E1008E7E8093E1008DE0F2
:103C80008093E200559A209A0E94010F82E480936B
:103C90000001809164008E7F8093640080917A009F
:103CA000806480937A0080917A0086FDFCCF009139
:103CB0007800109179000E94030DAB01BC01C8018E
:103CC000B0E0A0E0DC01992788276C017D01C40EDB
:103CD000D51EE61EF71EC701B601209164002160C3
:103CE00020936400611571058105910511F00E9412
:103CF00082301092D9021092D8021092DE020E94F5
:103D0000010F0E94570F80E80E944C0F8823A9F0F2
:103D10005C9885EA8EBD00000DB407FEFDCF5C9A6D
:103D20002E982F982D988091640080628093640073
:103D300081E083BF889513BEFCCF84E00E944C0FC6
:103D4000882309F448C02D9884E80E944C0F8823EA
:103D5000E1F00E94F20E88EC90E00E94F40E2F98A1
:103D600082E090E00E9420328F3F29F06FEF82E0E6
:103D700090E00E94283284EF91E00E94F40E2F9A86
:103D800084E80E944C0F8111FBCF84E10E944C0F0C
:103D90008823E1F00E94F20E88EC90E00E94F40E7D
:103DA0002E9882E090E00E942032882329F060E083
:103DB00082E090E00E94283284EF91E00E94F40EAD
:103DC0002E9A84E10E944C0F8111FBCF88EC90E089
:103DD0000E94F40EB2CF0E94F20E82E090E00E94A8
:103DE000FA158823E1F13E9A3F9A81E090E00E9423
:103DF000FA1581FF13C0082F0470302E82FD2E9813
:103E000001EF1FEFA8E0AA2EB12C80E40E944C0F16
:103E1000882341F12E9A2F9A0E94F20E82E390E0BD
:103E20000E94F40E0E94F90E8111F8CF8FB7F8941A
:103E30004091E0025091E1026091E2027091E30250
:103E40008FBF80916E02882309F4D0C010926E0259
:103E500080E090E0892B51F30E940000E7CF3E986C
:103E60003F98C3CF332029F00430110511F42E9A66
:103E70002F9881E00E94D707980117FF04C02227DE
:103E80003327201B310B27703327C80117FD0796F6
:103E9000F3E095958795FA95E1F717FF05C001972F
:103EA000A501421B530B9A01AC015695542F442790
:103EB0005795479542505D4FF12CE12C2501421A50
:103EC000530A8E3F6FEF960709F43EC0DA0170E0A7
:103ED00060E0F701E75DF74F4F013A01F0E86F0E40
:103EE000711C8F3F980781F0F401E60FF71FE491F2
:103EF000022E01C0EE0F0A94EAF75496FC915497F3
:103F0000EF2B5496EC93549721153105B9F0F40139
:103F1000E60FF71F24906301C60ED71EE22DF0E0D6
:103F2000042C02C0F595E7950A94E2F7FE87ED8729
:103F3000F6012488FD852F2AF601248A6F5F7F4FC2
:103F400011966835710569F60196F8E5EF0EF11CDA
:103F500040585F4F60EBE616F10409F0B2CF0E94C3
:103F6000570F8FE090E00E94F40E0F5F1F4F093152
:103F7000110509F04ACF332011F02F9A2D9880E9CE
:103F800091E00E94F40E0E94F20E81E090E00E9407
:103F9000FA1580FF43CF8AE090E00E94FA159FEF68
:103FA000980F9E3F08F03ACF22E330E03093710241
:103FB0002093700228E330E0309373022093720262
:103FC0000BE010E0682F84EA97E00E94C510C8015A
:103FD0000E94FA150F5F1F4F0131110599F70E94DA
:103FE000570F88EE93E00E94F40E18CF80916F0275
:103FF000942F981B892F90910001891748F48F5FA7
:10400000891708F025CF81E083BF889513BE20CFA4
:1040100081E080936E0240936F0280916C029091D8
:104020006D02019690936D0280936C0280917502EF
:10403000809374020E94F90E809375028091DE02D3
:104040008111FDC02091D8023091D902EEEFF2E04B
:1040500081118FEF00248193819381938193039445
:10406000D1F71092730210927202109271021092A4
:1040700070028091DC029091DD029093DB028093CC
:10408000DA021092DD021092DC022130310561F477
:104090008091D6029091D7024F9734F087E190E05B
:1040A0009093D9028093D8028091D8029091D9023E
:1040B0008831910508F0C5C4FC01EF59FF4D0C94FF
:1040C0009F347920BD20A121672167211D2246222E
:1040D0005F22C422482151235123512351235D23C0
:1040E00089232623A823A8234B244B244B244B2489
:1040F000B82441E65EE070E060E090E080E00E947D
:10410000D80941E65EE070E060E082E690E00E945F
:10411000D8098AE290E090937102809370028FE058
:1041200090E0909373028093720268E57EE084EAE7
:1041300097E00E94A10E87E68093950780939407ED
:104140008AE38093960761E57EE080E997E00E942C
:10415000A10E6FE37EE08CE697E00E94B81681E046
:1041600090E09093D5028093D4021092D3021092E3
:10417000D20241E050E060E04DC00E940119609120
:10418000D0027091D102CE0101960E941817CE0183
:1041900001960E94B313CE0101960E94171565E3A4
:1041A0007EE08CE697E00E94B8166AE27EE082E745
:1041B00097E00E94B8166FE17EE088E797E00E94E2
:1041C000B8166BE17EE08EE797E00E94B81680910A
:1041D000D0029091D102892B09F057C060E17EE0B6
:1041E00084E897E00E94B8166BE07EE08AE897E0EA
:1041F0000E94B81686E090E09093D5028093D40296
:104200001092D30281E08093D2024091D402509167
:10421000D50261E080E00E94EF0D2091D402309140
:10422000D50200E04091D2026091D3028091DA027F
:104230009091DB020E94511181E08093DE02C090D8
:10424000D802D090D902B8E1CB16D10408F09AC4B4
:10425000F601E35DFE4D0C949F343E253E253E2540
:104260003E253E253E253E25262C9A2B9A2B9A2B21
:104270009E2B9E2B9E2B9A2B9A2B9E2B1F2D1F2DF8
:104280001F2D1F2D1F2D1F2D9A2B84E090E0B4CFE2
:104290000E94011960E07EE0CE0101960E94E016C6
:1042A000CE0101960E94B313CE0101960E9417150C
:1042B00088EB92E00E94CB174091D4025091D50236
:1042C0006091D2028091D3020E94EF0DB5CF0E947F
:1042D00001198091D8029091D90266EF7DE0039791
:1042E00011F06BEE7DE0CE0101960E94E016CE014A
:1042F00001960E94B313CE0101960E94171580EA21
:1043000092E00E94CB174091D4025091D502609167
:10431000D2028091D3020E94EF0DE090DA02F09079
:10432000DB022091D4023091D50200E04091D2020C
:104330006091D302C7010E945111C7010E94A918C0
:104340007BCF0E94011961EE7DE0CE0107960E94AD
:10435000E0166091D0027091D102CE0101960E94C8
:104360001817BE016F5F7F4FCE0107960E94871618
:10437000CE0101960E9417151A8219821C821B8297
:104380001E821D826F8178856115710531F04B8524
:104390005C85CE0101960E944717CE0101960E94CE
:1043A000B313CE0101960E9417157CE6E72E77E045
:1043B000F72E70E060E08B010F5F1F4F8091D002FD
:1043C0009091D102681779070CF0B801CE010196DF
:1043D0000E941817BE016F5F7F4FC7010E94FC1536
:1043E000CE0101960E941715A6E0EA0EF11CB80155
:1043F0000530110501F71093D5020093D40281E036
:104400008093D3028093D20245E050E061E00E94A5
:10441000EF0D2091D4023091D50200E04091D202FC
:104420006091D3028091DA029091DB020E945111D7
:10443000CE0107960E941715FFCE0E94011966ED66
:104440007DE0CE0101960E94E016CE0101960E9409
:10445000B313CE0101960E9417156BEC7DE08CE63C
:1044600097E00E94B8166EEB7DE082E797E00E942D
:10447000B81682E090E09093D5028093D402109217
:10448000D3021092D20242E050E075CE0E94011990
:1044900069EB7DE0CE0101960E94E016CE01019607
:1044A0000E94B313CE0101960E9417156BEA7DE0BE
:1044B0008CE697E00E94B8166CE97DE0D6CF6DE8F7
:1044C0007DE08EE497E00E94B81662E87DE084E526
:1044D00097E00E94B81660919E0270919F02CE01F3
:1044E00001960E947217BE016F5F7F4F84E597E0CF
:1044F0000E948716CE0101960E9417156CE77DE099
:1045000084E597E00E945D166BE67DE08AE597E022
:104510000E94B8166DE57DE080E697E00E94B8162F
:1045200060919C0270919D02CE0101960E947217CB
:10453000BE016F5F7F4F80E697E00E948716CE0135
:1045400001960E94171584E090E090939B0280935F
:104550009A02109299020E94241382E48093950794
:104560008093940787E38093960769E97CE080E96C
:1045700097E00E94A10E83E490E00E941C1087E661
:1045800090E00E941C1058CE0E9433306B017C01D9
:1045900067E87CE08EE497E00E94B81660E87CE073
:1045A00084E597E00E94B81687E090E09093980227
:1045B0008093970283E090E090939B0280939A020D
:1045C00010929902C701B60122E030E040E050E0CD
:1045D0000E943632672B79F46BE77CE084E597E044
:1045E0000E945D1662E77CE08AE597E00E94B816BB
:1045F0000E94241321CE6BE67CE084E597E00E94C4
:104600005D1661E67CE08AE597E00E94B81680912D
:104610009C0290919D02039790939D0280939C022F
:10462000181619062CF363E57CE080E697E00E94FB
:10463000B81684E090E090939B0280939A0287E101
:1046400090E09093980280939702D2CF6BE47DE044
:104650008EE497E00E94B8166DE37DE084E597E074
:104660000E94B8166BE27DE08AE597E00E94B816DA
:1046700067E27DE080E697E00E94B81684E090E073
:1046800090939B0280939A02109299020E942413A5
:104690000E94101381E090E090939802809397021B
:1046A000CBCD0E9424138091D8029091D9020A9711
:1046B00009F4C2CD0E941013BFCD6DE571E08EE408
:1046C00097E00E94681764E771E084E597E00E9434
:1046D000681769E871E08AE597E00E94681760EA68
:1046E00071E080E697E00E94681767EB71E086E66C
:1046F00097E00E94681785E090E090939B0280937A
:104700009A0281E0809399020E9424138FE090E046
:10471000C3CF63E072E08EE497E00E9468176BEC11
:1047200071E084E597E00E9468176AED71E08AE520
:1047300097E00E94681783E090E090939B0280933B
:104740009A02109299020E94241387E190E0A4CF6C
:1047500060E27DE0419711F06AE17DE08EE497E050
:104760000E94B8166091950270919602CE01019652
:104770000E94E916BE016F5F7F4F8EE497E00E94B2
:104780008716CE0101960E94171566E27DE084E54A
:1047900097E00E94B81665E27DE08AE597E00E9406
:1047A000B8168091D8029091D9026BE07DE04197D4
:1047B00011F065E07DE080E697E00E94B81661E1C7
:1047C0007DE086E697E00E94B81685E090E0909341
:1047D0009B0280939A0281E0809399020E942413A5
:1047E000E0919502F0919602EE0FFF1FEE0FFF1F72
:1047F000E056FD4F20813181428153816091520703
:1048000070915307E5E0E69FC001E79F900D1124EA
:104810006AE070E00F960E94A8148091D8029091EF
:10482000D9024197E9F4209191023091920240918E
:104830009302509194026EE270E087E390E00E9450
:10484000A8140E94CB1461E07DE0CE0101960E9485
:10485000E016CE0101960E947514CE010196EACDB4
:1048600087E380939F0780939E078EE28093A00743
:10487000E0919502F0919602EE0FFF1FEE0FFF1FE1
:10488000E854FD4F40815181628173818AE997E04C
:104890000E941A14D6CF66EF7CE08331910559F05F
:1048A00069EE7CE08431910531F06BED7CE0459759
:1048B00011F06CEC7CE08EE497E00E94B81660E0AA
:1048C0007DE084E597E00E94B8166FEF7CE08AE512
:1048D00097E00E94B81680919702909198026BEB36
:1048E0007CE0059711F063EB7CE080E697E00E94A6
:1048F000B81663EC7CE086E697E00E94B81685E087
:1049000090E090939B0280939A0281E080939902B9
:104910000E94241380919702909198020597F9F4D0
:1049200020918D0230918E0240918F025091900221
:1049300065E270E082E390E00E94A8142091910269
:104940003091920240919302509194026EE270E095
:1049500087E390E00E94A8146FEA7CE076CF209174
:10496000890230918A0240918B0250918C02E0CFF3
:104970006091890270918A0280918B0290918C02E1
:104980000091910210919202209193023091940231
:10499000600F711F821F931F00918D0210918E0274
:1049A00020918F0230919002601B710B820B930B50
:1049B0000E94033120E030E04CEF51E40E943D338F
:1049C0000E9448340E94E5330E94AF336B0163E0DC
:1049D00072E08EE497E00E94681768EE71E084E56B
:1049E00097E00E94681765EF71E08AE597E00E9402
:1049F0006817B6016536710514F064E670E0CE0103
:104A000001960E947217BE016F5F7F4F8AE597E0A3
:104A10000E948716CE0101960E94171564E072E08D
:104A200080E697E00E9468171092990284E090E077
:104A300090939B0280939A02109298021092970290
:104A4000D7CD85E090E090937102809370029093AF
:104A500073028093720268EA7CE084EA97E00E9425
:104A6000A10E4091D8025091D902052E000C660B80
:104A7000770B84EA97E00E941A14DECB80E80E944C
:104A8000410F81111AC080E10E94410F811115C0B0
:104A900080E20E94410F811110C080E40E94410F0A
:104AA00081110BC088E00E94410F811106C084E093
:104AB0000E94410F882309F465C0A090D402B090F1
:104AC000D5027090D202E090DA02F090DB0201E0B1
:104AD0009501472D6091D302C7010E945111B50184
:104AE0000B2C000C880B990B0E94033120E030E066
:104AF00040E05FE30E9462311B012C0120E030E0C6
:104B0000A9010E943D3420E030E040E05FE387FDF2
:104B10003CC0C201B1010E94D1320E94AF338B016F
:104B200088248394912CE616F7061CF032E0832E3D
:104B3000912C80E10E94410F8823A1F1EFEFEE1A42
:104B4000FE0AEA14FB0434F5F092DB02E092DA028A
:104B5000E090DA02F090DB022091D4023091D5028D
:104B600000E04091D2026091D302C7010E9451112E
:104B70008091D8029091D9020397029718F4C70147
:104B80000E94A9180E94570F63C9C201B1010E9477
:104B9000D032C3CFF1E0AF1AB108B092DB02A092DD
:104BA000DA02D6CF80E80E94410F882371F001E03D
:104BB000E01AF108F092DB02E092DA02F7FEC8CFC9
:104BC0001092DB021092DA02C3CF80E40E94410F00
:104BD0008823D9F07720A9F08A94892891F4E00EEF
:104BE000F11EF092DB02E092DA028091DA029091FB
:104BF000DB028A159B050CF4ABCF41E0A41AB10887
:104C0000CCCF3FEFE31AF30AECCF80E20E94410FD2
:104C10008823B9F0772089F052E08516910469F471
:104C2000E01AF10AF092DB02E092DA028091DA02F5
:104C30009091DB0297FF8CCFC3CF61E0E61AF108B9
:104C4000F1CF88E00E94410F882309F45AC51092E1
:104C5000DE0283E0C816D10409F4BEC308F05AC0CE
:104C6000A1E0CA16D10409F486C0B2E0CB16D10483
:104C700009F4B0C0EF2809F06BCF81E090E0909389
:104C8000D9028093D80220ED37E040E050E0209335
:104C9000910230939202409393025093940288E8D9
:104CA00093E1A0E0B0E080938D0290938E02A093F8
:104CB0008F02B09390021092890210928A02109291
:104CC0008B0210928C021092D1021092D00210929C
:104CD00088021092870284E690E090938602809387
:104CE000850282E390E090939D0280939C02E8EB22
:104CF000F2E080ED92E011921192119211928E17D2
:104D00009F07C9F71092D7021092D60280E00E9446
:104D10001F151ECFE5E0CE16D10409F47DC408F4BA
:104D200022C406E0C016D10409F0A4CF86E090E0CA
:104D300090939802809397021092810210928202BF
:104D40001092830210928402E114F10409F4CAC49F
:104D5000EA94EF2809F0FCCE86E190E09093D90226
:104D60008093D8028091890290918A02A0918B024F
:104D7000B0918C0220C4D0929802C092970292E027
:104D8000E916F104F1F074F4E114F104B9F084E0EF
:104D900090E0EA94EF2809F0DBCE9093D90280935B
:104DA000D802D6CEE4E0EE16F10489F06CF086E08D
:104DB00090E005E0E016F10481F3CACE83E090E0D4
:104DC000ECCF89E090E0E9CF82E090E0E6CF85E0AB
:104DD00090E0E3CF8091D0029091D102E816F906DD
:104DE0001CF01FEFE11AF10AF092D102E092D0021A
:104DF00081E00E941F150E94333024E130E040E042
:104E000050E00E9436329B0141E050E050939802FE
:104E10004093970210929902FB013197E131F1051D
:104E200008F0D5C2EA5EF84D0C949F3427274E2730
:104E30006D27A027A027CB27CB27F8273F283F287F
:104E40003F28A028A028F42815294429B4296AEC71
:104E50007BE08EE497E00E94B8166CEB7BE084E583
:104E600097E00E94B81663EB7BE08AE597E00E942A
:104E7000B81683E090E090939B0280939A0222E020
:104E800030E040E050E02093B4023093B50240930C
:104E9000B6025093B7028AE090E07FCF62EA7BE0EF
:104EA0008EE497E00E94B81662E97BE084E597E023
:104EB0000E94B81682E090E090939B0280939A0241
:104EC0008AE790E0A0E0B0E08093AC029093AD025E
:104ED000A093AE02B093AF02DECF61E87BE08EE438
:104EE00097E00E94B81663E77BE084E597E00E94B4
:104EF000B81662E67BE08AE597E00E94B81669E59D
:104F00007BE080E697E00E94B81684E090E0909302
:104F10009B0280939A020E9433302EE734E040E0F7
:104F200050E00E9436326E5A7C4F8F4F9F4F6093F5
:104F3000A4027093A5028093A6029093A702ABCF20
:104F40006DE47BE08EE497E00E94B8166EE37BE0B0
:104F500084E597E00E94B81660E37BE08AE597E07D
:104F60000E94B81666E27BE080E697E00E94B816E1
:104F700084E090E090939B0280939A020E943330E9
:104F800029EA31E640E050E00E943632605B794B1E
:104F90008F4F9F4FCCCF66E17BE08EE497E00E947D
:104FA000B81664E07BE084E597E00E94B81661EFF4
:104FB0007AE08AE597E00E94B81683E090E090934B
:104FC0009B0280939A020E94333021E63AEE40E041
:104FD00050E00E9436326058774C8E4F9F4F60935E
:104FE000A0027093A1028093A2029093A30253CFD8
:104FF00061EE7AE08EE497E00E94B81662ED7AE006
:1050000084E597E00E94B81682E090E090939B02BE
:1050100080939A0260919102709192028091930222
:10502000909194020E94033120E030E040E450E48B
:105030000E943D336B017C0120E030E0A9010E9419
:105040003D3420E030E040E05FE387FD13C0C7015E
:10505000B6010E94D1320E94AF33660F771F881FBE
:10506000991F6093910270939202809393029093A0
:10507000940211CFC701B6010E94D032ECCFE8EB09
:10508000F2E090E080E04191519161917191840F43
:10509000951F42E0E03DF407B1F7C2970CF447C317
:1050A00082E090E02930310539F084E090E02A3048
:1050B000310511F085E090E090939F0280939E026D
:1050C00062EC7AE08EE497E00E94B8166DEB7AE02D
:1050D00084E597E00E94B81660919E0270919F024D
:1050E00061507109CE0101960E947217BE016F5F77
:1050F0007F4F84E597E00E948716CE0101960E94BB
:10510000171565EB7AE084E597E00E945D1668EA82
:105110007AE08AE597E00E94B8166DE97AE080E6C9
:1051200097E00E94B81684E090E090939B028093F1
:105130009A0287E090E09093980280939702ABCE1A
:105140008091910290919202A0919302B091940269
:10515000843F9140A105B1050CF4E9C20E94991267
:1051600005970CF4E4C20E94333023E030E040E0C5
:1051700050E00E9436326B016EE87AE08EE497E0F0
:105180000E94B81662E0C616D104C8F465E77AE05A
:10519000CD2811F066E67AE084E597E00E94B81623
:1051A00061E87AE08AE597E00E94B81683E090E033
:1051B00090939B0280939A028BE090E0EECD67E59E
:1051C0007AE084E597E00E94B81667E47AE08AE521
:1051D00097E00E94B8166EE37AE080E697E00E94BE
:1051E000B81684E090E0E4CF6CE27AE08EE497E0D9
:1051F0000E94B8166BE17AE084E597E00E94B81649
:1052000069E07AE08AE597E00E94B81666EF79E0F7
:1052100080E697E00E94B81684E090E090939B02AD
:1052200080939A028DE090E0B8CD809191029091A8
:105230009202A0919302B09194028C329140A10508
:10524000B1050CF474C263EE79E08EE497E00E943D
:10525000B81663ED79E084E597E00E94B81662EC39
:1052600079E08AE597E00E94B81667EB79E080E67E
:1052700097E00E94B81684E090E090939B028093A0
:105280009A028CE090E089CD0E94991208970CF464
:105290004EC20E94333027E030E040E050E00E94F0
:1052A00036328B010F5F1F4F0E94333026E030E013
:1052B00040E050E00E9436326B01FB01EE0FFF1F11
:1052C000EE0FFF1FE854FD4FA801012E000C660BE6
:1052D000770B80819181A281B381840F951FA61FD6
:1052E000B71F80839183A283B3836CEA79E08EE455
:1052F00097E00E94B816B801CE0101960E9472177D
:10530000BE016F5F7F4F8EE497E00E948716CE014B
:1053100001960E94171561EA79E084E597E00E9402
:10532000B816B601CE0101960E94E916BE016F5F64
:105330007F4F84E597E00E948716CE0101960E9478
:10534000171562E172E08AE597E00E94681764E24F
:1053500072E080E697E00E94681784E090E0909306
:105360009B0280939A0297CD62E372E08EE497E00D
:105370000E94681761E472E084E597E00E94681774
:1053800063E572E08AE597E00E94681762E672E0E2
:1053900080E697E00E94681784E090E090939B027B
:1053A00080939A020E94333027E232E040E050E0DE
:1053B0000E94363266507F4F8F4F9F4F6093A802F6
:1053C0007093A9028093AA029093AB0264CD50938C
:1053D000D9024093D802BCCB0E9499128C01D09282
:1053E0009802C0929702F0929602E09295021816E7
:1053F0001906F4F16DE47CE08EE497E00E94B816A3
:105400006CE47CE084E597E00E94B8166CE37CE0F5
:105410008AE597E00E94B81666E37CE080E697E0B4
:105420000E94B8166091950270919602CE01019685
:105430000E94E916BE016F5F7F4F80E697E00E94F1
:105440008716CE0101960E94171564E37CE080E682
:1054500097E00E945D1684E090E090939B02809319
:105460009A02109299028091D8029091D90263CE4B
:10547000F701EE0FFF1FEE0FFF1FE056FD4FC0803C
:10548000D180E280F38060919102709192028091CC
:105490009302909194026C157D058E059F0544F54D
:1054A0006EE27CE08EE497E00E94B8166DE27CE04C
:1054B00084E597E00E94B8166CE17CE08AE597E00D
:1054C0000E94B8166091950270919602CE010196E5
:1054D0000E94E916BE016F5F7F4F80E697E00E9451
:1054E000FC15CE0101960E9417156AE17CE0AFCF52
:1054F00021E130E03093D9022093D802109281024A
:105500001092820210928302109284020E94033150
:105510004B015C01C701B6010E9403319B01AC0144
:10552000C501B4010E943D330E94E5330E94AF33B0
:105530006093760270937702809378029093790259
:10554000012E000C220B330B06171707280739070B
:105550000CF0FECA00937602109377022093780233
:1055600030937902F5CA84E090E09093980280939A
:105570009702F0929602E0929502F701EE0FFF1F5C
:10558000EE0FFF1FE854FD4F80819181A281B3810E
:10559000181619061A061B06BCF422E130E03093F7
:1055A000D9022093D80210928102109282021092A6
:1055B0008302109284028093760290937702A093E4
:1055C0007802B0937902C4CA64E17CE08EE497E08B
:1055D0000E94B81663E17CE084E597E00E94B8166B
:1055E00060E07CE08AE597E00E94B8166091950241
:1055F00070919602CE0101960E94E916BE016F5F7E
:105600007F4F80E697E00E94FC15CE0101960E9434
:1056100017156EEF7BE01BCFD0929802C0929702D5
:1056200010928102109282021092830210928402E0
:10563000E114F10419F1EA94EF2809F089CA809184
:1056400080028823D1F162EF7BE08EE497E00E9434
:10565000B81663EE7BE084E597E00E94B8166CED27
:105660007BE08AE597E00E94B81683E090E0909393
:105670009B0280939A02109299020DCC83E190E0F4
:105680009093D9028093D802409191025091920256
:10569000609193027091940280918D0290918E029C
:1056A000A0918F02B0919002481759076A077B07B3
:1056B0000CF081CFDB01CA017ECF84E190E09093B2
:1056C000D9028093D802B8E8CB2EB3E1DB2EE12CCF
:1056D000F12CC0927602D0927702E0927802F0929A
:1056E000790236CA85E190E09093D9028093D8027E
:1056F0008091910290919202A0919302B0919402B4
:105700005ACF84E00E94410F882309F421CA12E095
:10571000C11AD10825E0C216D10408F019CA1092A6
:10572000DE020E94AF129093DD028093DC0281E0E2
:1057300090E033CB81E00E94EF1224CA80E00E9407
:10574000EF1281111FCA88E00E94410F882309F4DB
:1057500019CA1092DE028091D8029091D9028C3041
:10576000910509F44EC060F50B9709F00BCA8091C2
:105770008702909188020196909388028093870215
:105780008091910290919202A0919302B091940223
:1057900080599140A109B10980939102909392029E
:1057A000A0939302B0939402809185029091860217
:1057B0000597909386028093850281E090E041C036
:1057C0008D309105E1F1409709F0DCC9809191029B
:1057D00090919202A0919302B0919402885E9340BE
:1057E000A109B1098093910290939202A093930230
:1057F000B093940282E390E090939D0280939C0288
:10580000DCCF80918502909186020A969093860261
:10581000809385028091910290919202A0919302CF
:10582000B0919402885C9109A109B1098093910219
:1058300090939202A0939302B0939402BECF8EE015
:1058400090E09093D9028093D8029CC984E00E9492
:10585000410F8823E1F11092DE020E94333022E0F2
:1058600030E040E050E00E943632672B682B692B15
:10587000B9F460E979E08EE497E00E94B81665E833
:1058800079E084E597E00E94B81682E090E090937A
:105890009B0280939A021092990281E090E041C0AD
:1058A00065E779E08EE497E00E94B8166FE679E04C
:1058B00084E597E00E94B81682E090E090939B0206
:1058C00080939A021092990288E090E02AC088E0C2
:1058D0000E94410F882309F455C91092DE0280917D
:1058E000870290918802892B19F560E679E08EE4B1
:1058F00097E00E94B81662E579E084E597E00E949F
:10590000B81665E479E08AE597E00E94B81683E06E
:1059100090E090939B0280939A021092990287E004
:1059200090E090939802809397028AE090E089CF6C
:105930000E94333022E030E040E050E00E943632F6
:10594000672B682B692B49F464E479E08EE497E0D7
:105950000E94B81664E379E0ABCF80919E029091EB
:105960009F02019790939F0280939E02181619063A
:105970004CF463E379E08EE497E00E94B81662E2AB
:1059800079E096CF0E94333023EE34E040E050E0DF
:105990000E9436328B0102511D4F60E179E08EE4A6
:1059A00097E00E94B8166FEF78E084E597E00E94D8
:1059B000B816B801CE0101960E947217BE016F5F42
:1059C0007F4F84E597E00E948716CE0101960E94E2
:1059D00017156CEE78E08AE597E00E94B81669ED3D
:1059E00078E080E697E00E94B81684E090E090931B
:1059F0009B0280939A0281E080939902012E000C11
:105A0000220B330B8091910290919202A09193020C
:105A1000B0919402800F911FA21FB31F8093910237
:105A200090939202A0939302B0939402803B94408F
:105A3000A105B1050CF431CF80E190E072CF80E098
:105A40000E94EF1281119EC888E00E94410F8823B6
:105A500009F43FC18091D8029091D9028331910518
:105A600009F4BDC098F48131910509F47FC04297D3
:105A7000F1F11092DE020E94AF129093DD0280934A
:105A8000DC028091970290919802DBCE85319105DE
:105A900009F402C108F4CCC0469759F7409181023D
:105AA00050918202609183027091840280918902F8
:105AB00090918A02A0918B02B0918C02841B950B6D
:105AC000A60BB70B8093890290938A02A0938B0256
:105AD000B0938C028091910290919202A0919302D6
:105AE000B0919402840F951FA61FB71F36C08091F6
:105AF000950290919602209181023091820240910C
:105B0000830250918402880F991F880F991FFC010E
:105B1000E854FD4FC080D180E280F380C21AD30ADE
:105B2000E40AF50AC082D182E282F38280569D4F58
:105B3000DC016D917D918D919C910E948F3400913B
:105B40009102109192022091930230919402DC0113
:105B5000CB01800F911FA21FB31F809391029093DE
:105B60009202A0939302B093940283CF8091950206
:105B7000909196022091810230918202409183029D
:105B800050918402880F991F880F991FFC01E854D7
:105B9000FD4FC080D180E280F380C20ED31EE41E90
:105BA000F51EC082D182E282F38280569D4FFC01B5
:105BB00060817181828193810E948F340091910272
:105BC0001091920220919302309194026801790120
:105BD000C61AD70AE80AF90AD701C601BECF409112
:105BE00081025091820260918302709184028091BF
:105BF0008D0290918E02A0918F02B0919002841B31
:105C0000950BA60BB70B80938D0290938E02A093F9
:105C10008F02B09390028091910290919202A09194
:105C20009302B0919402841B950BA60BB70B95CFF2
:105C300040918102509182026091830270918402AE
:105C400080918D0290918E02A0918F02B09190026E
:105C5000840F951FA61FB71F80938D0290938E020D
:105C6000A0938F02B0939002809191029091920242
:105C7000A0919302B0919402840F951FA61FB71FA5
:105C80008093910290939202A0939302B093940216
:105C900081E080938002EDCE40918102509182029A
:105CA00060918302709184028091890290918A02AE
:105CB000A0918B02B0918C02840F951FA61FB71F75
:105CC0008093890290938A02A0938B02B0938C02F6
:105CD000A2CF8FB7F8944090E0025090E10260901C
:105CE000E2027090E3028FBF8091D8029091D902B6
:105CF0004197C12CD12C7601C394029728F07AE009
:105D0000C72ED12CE12CF12C80917C0290917D0248
:105D1000A0917E02B0917F0293018201081B190BB2
:105D20002A0B3B0B80917A0290917B0244EF51E069
:105D300060E070E08230910554F044E650E060E0AD
:105D400070E0853191051CF040E050E0BA01401749
:105D500051076207730710F00C94C2258436910531
:105D60000CF45EC05AE0852E912CA12CB12C8D37FD
:105D70009105BCF044E6842E912CA12CB12C8639DF
:105D800091057CF068EE862E63E0962EA12CB12C56
:105D90008F3A910534F030E1832E37E2932EA12C17
:105DA000B12C883E03E090072CF4019690937B027F
:105DB00080937A0280E80E944C0F882309F441C046
:105DC00040927C0250927D0260927E0270927F022D
:105DD0004091760250917702609178027091790239
:105DE0008091810290918202A0918302B0918402FD
:105DF0008A019B010C191D092E093F090817190773
:105E00002A073B0794F08C0D9D1DAE1DBF1D80938E
:105E1000810290938202A0938302B09384020DC00A
:105E2000812C912C54018394C0CF409381025093D4
:105E3000820260938302709384020E94CB140C94BC
:105E4000C22580E40E944C0F8823C9F140927C0255
:105E500050927D0260927E0270927F02AAE0B0E0D2
:105E6000A70196010E9455329B01AC01C501B40106
:105E70000E948F340091810210918202209183024E
:105E800030918402DC01CB01800F911FA21FB31F50
:105E90000091760210917702209178023091790278
:105EA000081719072A073B070CF0B1CF00938102AE
:105EB000109382022093830230938402BECF80E14C
:105EC0000E944C0F882319F140927C0250927D026F
:105ED00060927E0270927F02809181029091820294
:105EE000A0918302B09184028C159D05AE05BF057B
:105EF0002CF08C199D09AE09BF0989CF109281023F
:105F000010928202109283021092840296CF80E255
:105F10000E944C0F882351F140927C0250927D02E6
:105F200060927E0270927F02AAE0B0E0A701960123
:105F30000E9455329B01AC01C501B4010E948F340F
:105F4000009181021091820220918302309184029B
:105F500006171707280739078CF268017901C61A56
:105F6000D70AE80AF90AD701C60151CF10927C027C
:105F700010927D0210927E0210927F0210927B029C
:105F800010927A020C94C225CF93DF9386E697E0B5
:105F90000E94171580E697E00E9417158AE597E0A2
:105FA0000E94171584E597E00E9417158EE497E08C
:105FB0000E941715C0E9D7E02697CE010E94171559
:105FC00087E0CC36D807C1F7DF91CF9108958F9243
:105FD0009F92AF92BF92CF92DF92EF92FF92CF93B8
:105FE000DF93EC01688179818A819B81611571055C
:105FF0008105910521F464E279ED8BE597E02DE1CF
:1060000033EF41E050E00E94363249015A019B01D2
:10601000AC01A7EAB1E40E9455326B017C01ACEE01
:10602000B4EFA50194010E946332C60ED71EE81E8C
:10603000F91EF7FE06C081E0C81AD108E10880E821
:10604000F80AC882D982EA82FB82C701B6019F772B
:10605000DF91CF91FF90EF90DF90CF90BF90AF9006
:106060009F908F9008958F929F92AF92BF92CF9200
:10607000DF92EF92FF9260910D0170910E0180917D
:106080000F0190911001611571058105910521F4B1
:1060900064E279ED8BE597E02DE133EF41E050E0EC
:1060A0000E94363249015A019B01AC01A7EAB1E4D2
:1060B0000E9455326B017C01ACEEB4EFA501940156
:1060C0000E946332C60ED71EE81EF91EF7FE06C0F8
:1060D00081E0C81AD108E10880E8F80AC0920D01F1
:1060E000D0920E01E0920F01F0921001C701B601AB
:1060F0009F77FF90EF90DF90CF90BF90AF909F90F1
:106100008F90089560930D0170930E0180930F019D
:10611000909310010895FB01DC0105900D92002081
:10612000E1F70895FC0105900020E9F7809590952E
:106130008E0F9F1F0895BB274A3031F4992322F414
:10614000BDE2909581959F4F0C94D830BB272A30A3
:1061500051F4992342F4BDE2909580957095619534
:106160007F4F8F4F9F4F0C94B630BB27FA01A62F5D
:106170006217710581059105330B30FB66F0AA2784
:10618000660F771F881F991FAA1FA21710F0A21B66
:1061900063953850A9F7A05DAA3308F0A95DA193D3
:1061A00036F7B111B1931082CA010C94F130BB27BC
:1061B000FB015527AA27880F991FAA1FA41710F0C3
:1061C000A41B83955051B9F7A05DAA3308F0A95DCF
:1061D000A193009779F7B111B1931192CB010C946F
:1061E000F130DC01FC01672F71917723E1F73297E1
:1061F00004C07C916D9370836291AE17BF07C8F3A2
:106200000895E89409C097FB3EF4909580957095A9
:1062100061957F4F8F4F9F4F9923A9F0F92F96E9F2
:10622000BB279395F695879577956795B795F11167
:10623000F8CFFAF4BB0F11F460FF1BC06F5F7F4F04
:106240008F4F9F4F16C0882311F096E911C0772316
:1062500021F09EE8872F762F05C0662371F096E81F
:10626000862F70E060E02AF09A95660F771F881FEE
:10627000DAF7880F9695879597F90895990F000892
:10628000550FAA0BE0E8FEEF16161706E807F90708
:10629000C0F012161306E407F50798F0621B730BA3
:1062A000840B950B39F40A2661F0232B242B252B24
:1062B00021F408950A2609F4A140A6958FEF811DC7
:1062C000811D08950E9475310C94E6310E94D831E9
:1062D00038F00E94DF3120F0952311F00C94CF317B
:1062E0000C94D53111240C941A320E94F73170F3BA
:1062F000959FC1F3950F50E0551F629FF001729F6B
:10630000BB27F00DB11D639FAA27F00DB11DAA1F79
:10631000649F6627B00DA11D661F829F2227B00DC6
:10632000A11D621F739FB00DA11D621F839FA00D51
:10633000611D221F749F3327A00D611D231F849FA1
:10634000600D211D822F762F6A2F11249F575040F8
:106350009AF0F1F088234AF0EE0FFF1FBB1F661F73
:10636000771F881F91505040A9F79E3F510580F03C
:106370000C94CF310C941A325F3FE4F3983ED4F37F
:10638000869577956795B795F795E7959F5FC1F7E0
:10639000FE2B880F911D9695879597F9089597F98B
:1063A0009F6780E870E060E008959FEF80EC0895BB
:1063B00000240A94161617061806090608950024E4
:1063C0000A9412161306140605060895092E03945E
:1063D000000C11F4882352F0BB0F40F4BF2B11F4D2
:1063E00060FF04C06F5F7F4F8F4F9F4F089557FD31
:1063F0009058440F551F59F05F3F71F04795880F33
:1064000097FB991F61F09F3F79F0879508951216C9
:1064100013061406551FF2CF4695F1DF08C0161675
:1064200017061806991FF1CF869571056105089426
:106430000895E894BB2766277727CB0197F908953D
:10644000F999FECF92BD81BDF89A992780B508953C
:10645000262FF999FECF1FBA92BD81BD20BD0FB680
:10646000F894FA9AF99A0FBE01960895052E97FBB3
:106470001EF400940E944D3257FD07D00E949F32B7
:1064800007FC03D04EF40C944D3250954095309556
:1064900021953F4F4F4F5F4F089590958095709590
:1064A00061957F4F8F4F9F4F08950E94C132A59FE6
:1064B000900DB49F900DA49F800D911D11240895FF
:1064C000B7FF0C9455320E945532821B930B0895EE
:1064D0002F923F924F925F926F927F928F929F92F4
:1064E000AF92BF92CF92DF92EF92FF920F931F93E2
:1064F000CF93DF93CDB7DEB7CA1BDB0B0FB6F89493
:10650000DEBF0FBECDBF09942A88398848885F84D2
:106510006E847D848C849B84AA84B984C884DF8043
:10652000EE80FD800C811B81AA81B981CE0FD11D27
:106530000FB6F894DEBF0FBECDBFED010895A1E206
:106540001A2EAA1BBB1BFD010DC0AA1FBB1FEE1FED
:10655000FF1FA217B307E407F50720F0A21BB30B38
:10656000E40BF50B661F771F881F991F1A9469F7B4
:1065700060957095809590959B01AC01BD01CF0110
:106580000895A29FB001B39FC001A39F700D811D0C
:106590001124911DB29F700D811D1124911D08952C
:1065A0005058BB27AA270E94E8320C94E6310E947B
:1065B000D83138F00E94DF3120F039F49F3F19F4D0
:1065C00026F40C94D5310EF4E095E7FB0C94CF3112
:1065D000E92F0E94F73158F3BA176207730784074F
:1065E000950720F079F4A6F50C9419320EF4E09595
:1065F0000B2EBA2FA02D0B01B90190010C01CA017D
:10660000A0011124FF27591B99F0593F50F4503E27
:1066100068F11A16F040A22F232F342F4427585F19
:10662000F3CF469537952795A795F0405395C9F731
:106630007EF41F16BA0B620B730B840BBAF09150E9
:10664000A1F0FF0FBB1F661F771F881FC2F70EC088
:10665000BA0F621F731F841F48F48795779567955B
:10666000B795F7959E3F08F0B0CF9395880F08F047
:106670009927EE0F9795879508950E9451330C94B2
:10668000E6310E94DF3158F00E94D83140F029F401
:106690005F3F29F00C94CF3151110C941A320C94B5
:1066A000D5310E94F73168F39923B1F3552391F363
:1066B000951B550BBB27AA2762177307840738F071
:1066C0009F5F5F4F220F331F441FAA1FA9F335D0CE
:1066D0000E2E3AF0E0E832D091505040E695001C82
:1066E000CAF72BD0FE2F29D0660F771F881FBB1F3C
:1066F000261737074807AB07B0E809F0BB0B802D1A
:10670000BF01FF2793585F4F3AF09E3F510578F045
:106710000C94CF310C941A325F3FE4F3983ED4F3DB
:10672000869577956795B795F7959F5FC9F7880F19
:10673000911D9695879597F90895E1E0660F771F6B
:10674000881FBB1F621773078407BA0720F0621BFC
:10675000730B840BBA0BEE1F88F7E09508950E9427
:10676000B6336894B1110C941A3208950E94FF3127
:1067700088F09F5798F0B92F9927B751B0F0E1F002
:10678000660F771F881F991F1AF0BA95C9F714C0B2
:10679000B13091F00E941932B1E008950C94193291
:1067A000672F782F8827B85F39F0B93FCCF38695EB
:1067B00077956795B395D9F73EF490958095709548
:1067C00061957F4F8F4F9F4F08950E94253490F021
:1067D0009F3748F4911116F00C941A3260E070E083
:1067E00080E89FEB089526F41B16611D711D811D25
:1067F0000C94FC330C941734882371F4772321F024
:106800009850872B762F07C0662311F499270DC067
:106810009051862B70E060E02AF09A95660F771F02
:10682000881FDAF7880F9695879597F908959F3F07
:1068300031F0915020F4879577956795B795880F3B
:10684000911D9695879597F908950E94FF31A0F0C4
:10685000BEE7B91788F4BB279F3860F41616B11D40
:10686000672F782F8827985FF7CF8695779567955C
:10687000B11D93959639C8F308950E943E3108F4EE
:106880008FEF089519F416F40C94D5310C94173445
:106890000E94FF31B8F39923C9F3B6F39F57550B04
:1068A00087FF0E9488340024A0E640EA90018058C7
:1068B0005695979528F4805C660F771F881F20F007
:1068C00026173707480730F4621B730B840B202907
:1068D00031294A2BA69517940794202531254A275C
:1068E00058F7660F771F881F20F0261737074807CD
:1068F00030F4620B730B840B200D311D411DA095EC
:1069000081F7B901842F9158880F9695879508953E
:1069100091505040660F771F881FD2F70895DB0112
:106920008F939F930E945532BF91AF91A29F800D8C
:10693000911DA39F900DB29F900D11240895EE0F0D
:10694000FF1F0590F491E02D09940F931F93CF93AF
:10695000DF938230910510F482E090E0E091AA0785
:10696000F091AB0730E020E0B0E0A0E0309799F480
:106970002115310509F44AC0281B390B2430310593
:10698000D8F58A819B816115710589F1FB0193839B
:106990008283FE0111C04081518102811381481719
:1069A0005907E0F04817590799F4109761F01296CB
:1069B0000C93129713961C933296CF01DF91CF91CF
:1069C0001F910F9108950093AA071093AB07F4CF7E
:1069D0002115310551F04217530738F0A901DB01A9
:1069E0009A01BD01DF01F801C1CFEF01F9CF90930A
:1069F000AB078093AA07CDCFFE01E20FF31F81936F
:106A000091932250310939832883D7CF2091A80749
:106A10003091A907232B41F42091130130911401E7
:106A20003093A9072093A8072091110130911201FA
:106A30002115310541F42DB73EB740911501509114
:106A40001601241B350BE091A807F091A907E21766
:106A5000F307A0F42E1B3F0B2817390778F0AC0181
:106A60004E5F5F4F2417350748F04E0F5F1F50935E
:106A7000A9074093A807819391939FCFF0E0E0E0AE
:106A80009CCFCF93DF930097E9F0FC0132971382FC
:106A90001282A091AA07B091AB07ED0130E020E08F
:106AA0001097A1F420813181820F931F2091A807B4
:106AB0003091A9072817390709F061C0F093A90799
:106AC000E093A807DF91CF910895EA01CE17DF0781
:106AD000E8F54A815B819E0141155105B1F7E90155
:106AE000FB83EA8349915991C40FD51FEC17FD0729
:106AF00061F4808191810296840F951FE901998349
:106B00008883828193819B838A83F0E0E0E0129600
:106B10008D919C9113970097B9F52D913C91119708
:106B2000CD010296820F931F2091A8073091A907EB
:106B30002817390739F6309751F51092AB071092A4
:106B4000AA07B093A907A093A807BCCFD383C28399
:106B500040815181840F951FC817D90761F44E5F9A
:106B60005F4F88819981480F591F518340838A81E3
:106B70009B81938382832115310509F0B0CFF09377
:106B8000AB07E093AA079ECFFD01DC01C0CF1382C3
:106B90001282D7CFB0E0A0E0E0EDF5E30C946A32CA
:106BA0008C01009751F4CB010E94A5348C01C801DF
:106BB000CDB7DEB7E0E10C948632FC01E60FF71F9B
:106BC0009C0122503109E217F30708F49DC0D90156
:106BD000CD91DC911197C617D70798F0C530D10534
:106BE00030F3CE0104978617970708F3C61BD70B1F
:106BF0002297C193D1936D937C93CF010E9441352D
:106C0000D6CF5B01AC1ABD0A4C018C0E9D1EA09123
:106C1000AA07B091AB07512C412CF12CE12C109715
:106C200031F58091A8079091A9078815990509F079
:106C30005CC04616570608F058C08091110190912B
:106C40001201009741F48DB79EB740911501509104
:106C50001601841B950BE817F90708F055C0F0934F
:106C6000A907E093A807F90171836083A0CF8D91F4
:106C70009C91119712966C90129713967C90139793
:106C8000A815B90559F56C0142E0C40ED11CCA140F
:106C9000DB0420F1AC014A195B09DA011296159761
:106CA00080F06282738251834083D9016D937C931B
:106CB000E114F10471F0D7011396FC93EE9312974F
:106CC00076CF22968C0F9D1FF90191838083F3016B
:106CD000EFCFF093AB07E093AA0769CF48165906A8
:106CE00008F42C017D01D3019ACFCB010E94A53479
:106CF0007C01009749F0AE01B8010E948736C801B7
:106D00000E944135870153CF10E000E050CFFB01D6
:106D1000DC0102C001900D9241505040D8F7089517
:106D2000FB01DC0101900D920020E1F7089517E0CE
:106D3000CCEAD7E004C0FE010E949F342196CD3AF0
:086D4000D107C9F7F894FFCF59
:106D480010FFFFFFFF00E10000000000000100004D
:106D5800000000AC07800000C18081000000000036
:106D68000000F00B5B0D110C060C570C150C330CC6
:106D7800000000004B12C50EBE13E00D000000001D
:106D8800FD11C50EBE13E00D00000000C510C50EB4
:106D9800BE13E00D596F75206F776E2000596F751F
:106DA8002068616C6C7563696E617465206F6E2014
:106DB8007468650077696C646573742074726970AF
:106DC800206F6620796F7572006C6966652C207378
:106DD80074756D626C65206F6E746F2074686500E1
:106DE80073756277617920747261636B732C2061AB
:106DF8006E642067657400637265616D6564206206
:106E080079206120747261696E2E002020204A75F5
:106E1800737420736179206E6F0020202020746FB6
:106E28002064727567732E00202047616D65206F9E
:106E380076657221002020596F75722073636F7216
:106E4800653A200020206F7574206F66203130303D
:106E58002E006F6E2061206465616420647564652E
:106E680020696E00746865207375627761792121E5
:106E78002100546865206D61726B657420686173C8
:106E8800006265656E20666C6F6F64656420776963
:106E9800746800636865617020686F6D656D616412
:0C6EA80065006163696421212121000064
:00000001FF
